:020000040000fa
:080000000002040000000000f2
:020000040000fa
:04000800f4040000fc
:020000040000fa
:04000c00f4040000f8
:020000040000fa
:04001000f4040000f4
:020000040000fa
:04001400f4040000f0
:020000040000fa
:04001800f4040000ec
:020000040000fa
:04001c00f4040000e8
:020000040000fa
:04002000f4040000e4
:020000040000fa
:04002400f4040000e0
:020000040000fa
:04002800d4020000fe
:020000040000fa
:04002c00f4040000d8
:020000040000fa
:04003000f8020000d2
:020000040000fa
:04003400f4040000d0
:020000040000fa
:04003800f4040000cc
:020000040000fa
:04003c00f4040000c8
:020000040000fa
:040040003003000089
:020000040000fa
:04004400f4040000c0
:020000040000fa
:04004800f4040000bc
:020000040000fa
:04004c00f4040000b8
:020000040000fa
:04005000b6040000f2
:020000040000fa
:04005400f4040000b0
:020000040000fa
:04005800f4040000ac
:020000040000fa
:04005c00f4040000a8
:020000040000fa
:04006000f4040000a4
:020000040000fa
:04006400f4040000a0
:020000040000fa
:04006800f40400009c
:020000040000fa
:04006c00f404000098
:020000040000fa
:04007000f404000094
:020000040000fa
:04007400f404000090
:020000040000fa
:0400780098030000e9
:020000040000fa
:04007c00f404000088
:020000040000fa
:04008000f404000084
:020000040000fa
:04008400f404000080
:020000040000fa
:04008800f40400007c
:020000040000fa
:04008c00f404000078
:020000040000fa
:04009000f404000074
:020000040000fa
:04009400f404000070
:020000040000fa
:04009800f40400006c
:020000040000fa
:04009c00f803000065
:020000040000fa
:0400a000f404000064
:020000040000fa
:0400a400f404000060
:020000040000fa
:0400a800f40400005c
:020000040000fa
:0400ac00f404000058
:020000040000fa
:0400b000f404000054
:020000040000fa
:0400b400f404000050
:020000040000fa
:0400b800f40400004c
:020000040000fa
:0400bc00f404000048
:020000040000fa
:0400c000f404000044
:020000040000fa
:0400c400f404000040
:020000040000fa
:0400c800f40400003c
:020000040000fa
:0400cc00f404000038
:020000040000fa
:0400d000f404000034
:020000040000fa
:0400d400f404000030
:020000040000fa
:0400d800f40400002c
:020000040000fa
:0400dc00f404000028
:020000040000fa
:0400e000f404000024
:020000040000fa
:0400e400f404000020
:020000040000fa
:0400e800f40400001c
:020000040000fa
:0400ec00f404000018
:020000040000fa
:0400f000f404000014
:020000040000fa
:0400f400f404000010
:020000040000fa
:0400f800f40400000c
:020000040000fa
:0400fc00f404000008
:020000040000fa
:04010000f404000003
:020000040000fa
:04010400f4040000ff
:020000040000fa
:04010800f4040000fb
:020000040000fa
:04010c00f4040000f7
:020000040000fa
:04011000f4040000f3
:020000040000fa
:04011400f4040000ef
:020000040000fa
:04011800f4040000eb
:020000040000fa
:04011c00f4040000e7
:020000040000fa
:04012000f4040000e3
:020000040000fa
:04012400f4040000df
:020000040000fa
:04012800f4040000db
:020000040000fa
:04012c00f4040000d7
:020000040000fa
:04013000f4040000d3
:020000040000fa
:04013400f4040000cf
:020000040000fa
:04013800f4040000cb
:020000040000fa
:04013c00f4040000c7
:020000040000fa
:04014000f4040000c3
:020000040000fa
:04014400f4040000bf
:020000040000fa
:04014800f4040000bb
:020000040000fa
:04014c00f4040000b7
:020000040000fa
:04015000f4040000b3
:020000040000fa
:04015400f4040000af
:020000040000fa
:04015800f4040000ab
:020000040000fa
:04015c00f4040000a7
:020000040000fa
:04016000f4040000a3
:020000040000fa
:04016400f40400009f
:020000040000fa
:04016800f40400009b
:020000040000fa
:04016c00f404000097
:020000040000fa
:04017000f404000093
:020000040000fa
:04017400f40400008f
:020000040000fa
:04017800f40400008b
:020000040000fa
:04017c00f404000087
:020000040000fa
:04018000f404000083
:020000040000fa
:04020800f4040000fa
:020000040000fa
:04020c00f4040000f6
:020000040000fa
:04021000f4040000f2
:020000040000fa
:04021400f4040000ee
:020000040000fa
:04021800f4040000ea
:020000040000fa
:04021c00f4040000e6
:020000040000fa
:04022000f4040000e2
:020000040000fa
:04022400f4040000de
:020000040000fa
:04022800f4040000da
:020000040000fa
:04022c00f4040000d6
:020000040000fa
:04023000f4040000d2
:020000040000fa
:04023400f4040000ce
:020000040000fa
:04023800f4040000ca
:020000040000fa
:04023c00f4040000c6
:020000040000fa
:04024000f4040000c2
:020000040000fa
:04024400f4040000be
:020000040000fa
:04024800f4040000ba
:020000040000fa
:04024c00f4040000b6
:020000040000fa
:04025000f4040000b2
:020000040000fa
:04025400f4040000ae
:020000040000fa
:04025800f4040000aa
:020000040000fa
:04025c00f4040000a6
:020000040000fa
:04026000f4040000a2
:020000040000fa
:04026400f40400009e
:020000040000fa
:04026800f40400009a
:020000040000fa
:04026c00f404000096
:020000040000fa
:04027000f404000092
:020000040000fa
:04027400f40400008e
:020000040000fa
:04027800f40400008a
:020000040000fa
:04027c00f404000086
:020000040000fa
:04028000f404000082
:020000040000fa
:04028400f40400007e
:020000040000fa
:04028800f40400007a
:020000040000fa
:04028c00f404000076
:020000040000fa
:04029000f404000072
:020000040000fa
:04029400f40400006e
:020000040000fa
:04029800f40400006a
:020000040000fa
:04029c00f404000066
:020000040000fa
:0402a000f404000062
:020000040000fa
:0402a400f40400005e
:020000040000fa
:0402a800f40400005a
:020000040000fa
:0402ac00f404000056
:020000040000fa
:0402b000f404000052
:020000040000fa
:0402b400f40400004e
:020000040000fa
:0402b800f40400004a
:020000040000fa
:0402bc00f404000046
:020000040000fa
:0402c000f404000042
:020000040000fa
:0402c400f40400003e
:020000040000fa
:0402c800f40400003a
:020000040000fa
:0402cc00f404000036
:020000040000fa
:0402d000f404000032
:020000040000fa
:0402d400f40400002e
:020000040000fa
:0402d800f40400002a
:020000040000fa
:0402dc00f404000026
:020000040000fa
:0402e000f404000022
:020000040000fa
:0402e400f40400001e
:020000040000fa
:0402e800f40400001a
:020000040000fa
:0402ec00f404000016
:020000040000fa
:0402f000f404000012
:020000040000fa
:0402f400f40400000e
:020000040000fa
:0402f800f40400000a
:020000040000fa
:0402fc00f404000006
:020000040000fa
:04030000f404000001
:020000040000fa
:04030400f4040000fd
:020000040000fa
:04030800f4040000f9
:020000040000fa
:04030c00f4040000f5
:020000040000fa
:04031000f4040000f1
:020000040000fa
:04031400f4040000ed
:020000040000fa
:04031800f4040000e9
:020000040000fa
:04031c00f4040000e5
:020000040000fa
:04032000f4040000e1
:020000040000fa
:04032400f4040000dd
:020000040000fa
:04032800f4040000d9
:020000040000fa
:04032c00f4040000d5
:020000040000fa
:04033000f4040000d1
:020000040000fa
:04033400f4040000cd
:020000040000fa
:04033800f4040000c9
:020000040000fa
:04033c00f4040000c5
:020000040000fa
:04034000f4040000c1
:020000040000fa
:04034400f4040000bd
:020000040000fa
:04034800f4040000b9
:020000040000fa
:04034c00f4040000b5
:020000040000fa
:04035000f4040000b1
:020000040000fa
:04035400f4040000ad
:020000040000fa
:04035800f4040000a9
:020000040000fa
:04035c00f4040000a5
:020000040000fa
:04036000f4040000a1
:020000040000fa
:04036400f40400009d
:020000040000fa
:04036800f404000099
:020000040000fa
:04036c00f404000095
:020000040000fa
:04037000f404000091
:020000040000fa
:04037400f40400008d
:020000040000fa
:04037800f404000089
:020000040000fa
:04037c00f404000085
:020000040000fa
:04038000f404000081
:020000040000fa
:10040000effe20000e7f22000e0188000000000099
:10041000000020000000e000020032000001200087
:100420002002880014000700e60107000000e00039
:1004300003003a0080a223000100200002003700e0
:100440000000200001002000810f70000100320038
:1004500014000700000020000000e000020032004d
:100460000000020000000000b4390200000000009b
:100470000040da000000fe004440a9000092200085
:100480000000e0000300320000002000a00188000e
:100490004440a800000006008a1f78008b1f7800e7
:1004a0000000060091018800800478000000eb0045
:1004b0001a003700e284440032a0b4009905ba0063
:1004c000e284440032a0b4009906ba00e2844400f9
:1004d00032a0b4000006eb00476fde00fd07b2005b
:1004e000636ce10003003a00ebff07000000eb0043
:1004f0000a003700606ce10004003a00005deb0088
:100500008b05e900fdff3e00040037006168e10053
:10051000010032000086eb000b00070019c7ba008b
:100520001905ba000e04e00003003a000a00e000da
:10053000e0ff3a0000000600fe07b2009e018800be
:100540008a047800f5ff3700395dba008b05e900b1
:100550000c003200295dba008b05e900080032006a
:100560000c00e00003003a00e284440032a0b40032
:10057000f5ff370019ddba008b05e900faff3a00f4
:100580008904e800e184440032a0b40000000600c1
:10059000000000000000000000000000000000005b
:1005a0000000000000000000801f78003400f80008
:1005b00000002000a001880000012000b041880058
:1005c0003828ef00a221ef0080ff2f009a01b6002b
:1005d0003000b300d00c880094c0a8009400a9009b
:1005e0008400a9003400f9004f00780000400600a4
:1005f000809fbe003400f80000002000a0018800a9
:100600003208e2000d003400a1418000e18060006a
:10061000c508dd00601680000050a1000080700059
:10062000601688003428d5003228ed008440a900e7
:100630003400f9004f00be0000400600cca2a80024
:100640009440a9003428d5003228ed008440a90048
:100650003400f9004f00be0000400600f7ff3700ed
:10066000809fbe00829fbe003400f8000000200082
:10067000a0018800cae2ab000100320039e8a800fe
:100680003628ed003608e2001b003a0094c0a900ad
:1006900080ff2f009a21b60010438000f107200050
:1006a000810f50000d003c000000e800104388005e
:1006b00000438000e300400081804000e28520008c
:1006c000c341800003b178000000e800f107280072
:1006d0000100600010003300004388009400a8006f
:1006e00084c0a9008400a9003400f9004f01be00b5
:1006f0004f00be00004006003828d50084c0a90085
:100700008400a9003400f9004f01be004f00be0074
:1007100000400600f8ff37000000e90001f82f0054
:10072000008070000000e80000438800ebff370005
:10073000809fbe00829fbe003400f80000002000b1
:10074000a0018800d2e2ab00010032005108a800ed
:100750004e28ed004e08e20018003a007063800059
:10076000f1072000810f50000d003c000000e80060
:100770007063880060638000e30040008180400077
:10078000a2c620008342800003b178000000e80088
:10079000f1072800010060000f003300606388004b
:1007a000b0002000704288008680a9003400f90063
:1007b0004f01be004f00be00004006005028d5008b
:1007c0008680a9003400f9004f01be004f00be0032
:1007d00000400600f9ff37000000e90001f82f0093
:1007e000008070000000e80060638800ecff3700c4
:1007f000809fbe00829fbe003400f80000002000f1
:10080000a00188004a08e20022003a00cd02a900b7
:10081000cd02a800cd02a900d322ab000100320016
:100820004528a8004228ed004208e20042003a00b4
:10083000a06b8000f1072000810f50000d003c00ec
:100840000000e800a06b8800906b8000e30040008f
:100850008180400002d720002342800003b178004d
:100860000000e800f10728000100600039003300b3
:10087000906b8800b0002000104288004428ef00f0
:1008800087a0a9003400f9004f01be004f00be0050
:10089000004006004608e2001d003a0097a0a900ab
:1008a00041428000e1806000c908dd00a0168000a0
:1008b0000090a10000807000a0168800d302ab0059
:1008c000feff3a000000000000000000d122a80056
:1008d000d102a800d322ab00feff3a00b0002000f6
:1008e000104288004428ef004a28ef0097a0a80093
:1008f0004828d5004628ed0087a0a9003400f9005b
:100900004f01be004f00be0000400600e1ff37006f
:1009100041428000e1806000c908dd00a01680002f
:100920000090a10000807000a01688004828d50023
:100930004628ed00f0ff37004428d50087a0a90025
:100940003400f9004f01be004f00be000040060019
:10095000d0ff37000000e90001f82f000080700090
:100960000000e800906b8800c2ff3700809fbe0047
:10097000821f78003400f80000002000a0018800e9
:10098000421280008540a90010788000f107200005
:10099000810f50000a003c000000e8001078880039
:1009a0000078800041f02000827078000000e800ac
:1009b000f10728000100600005003300007888007e
:1009c0003400f9004f0178004f00be0000400600df
:1009d0000000e90001f82f00008070000000e8002e
:1009e00000788800f6ff37000040da000000fe00c3
:1009f0000a00fa0011002000b1bf9f00c0bf9f0095
:100a00006a805700500607004fb897000080fa0030
:100a1000000006000a00fa00e20f500034003e0019
:100a2000507f8000e10f500003003200e20f5000c1
:100a300011003a000c003700032220000300e00000
:100a400001003a000040da002002e2000200350016
:100a50002822ef0021e2a8002342ab000d003a005b
:100a60002342a8000b003700032320000300e0000e
:100a700001003a000040da003002e20002003500d6
:100a80003822ef0031e2a8003342ab0001003a0007
:100a90003342a800820178000b0037003102fb00ce
:100aa000e10f500004003a002322ab00feff3a00a1
:100ab00024118800030037003322ab00feff3a0008
:100ac000a41188008301e9000300e000f3ff3a006d
:100ad000e10f500003003a002302ab00feff32009a
:100ae0000b0037003302ab00feff32000800370076
:100af00033002000b3bf9f00c0bf9f00d1bf9f0045
:100b0000e2bf9f006a805700110607006fb9970087
:100b1000020078000080fa00000006000a00fa00d7
:100b200051002000b1bf9f00c0bf9f006a805700e6
:100b3000090607005fb897000080fa000000060071
:100b4000889fbe0080047800607f80000000e00085
:100b500004003a000e0007000084eb000000e000f3
:100b600008003500687f80000900e00005003200c1
:100b700009004400060007000000e00001003d00fd
:100b80000084eb00080078004f04be00000006005f
:100b9000800078000100e00003003a00000020001f
:100ba000607f8800000005000080eb00020020004c
:100bb000828f500002003e00617f88000000eb0041
:100bc0000000060000000500889fbe008a9fbe004e
:100bd0008c9fbe008e1f780000067800010478000c
:100be00002007800830478000881b90002077800c9
:100bf0000200e000420032000800e0004100320044
:100c000082057800c900900069009000808f500034
:100c10000400390009007800500007000000e000df
:100c20002900350000402000190060000a00320051
:100c30000b017800a10020000c00780036000700ae
:100c4000800678000d00e000060032006105160005
:100c50000a854600040037000b0578008006eb008b
:100c6000010037000b05780049009000e900900072
:100c7000808050008a8f500002003100010578000a
:100c80008006eb000a0178008c0078002c00070039
:100c90008a855500490090000a004000c004980071
:100ca0000d00e0000400320009007800d5000700c4
:100cb0000000e00004003a000b00e00002003200f7
:100cc0000a064600cfff37000080200019006000b0
:100cd0000200320009007800ca00070000c02000ae
:100ce000190060000200320049009000e004980002
:100cf0008b055700110009008885d80001003700d6
:100d00000000eb004f0778004f06be004f05be0005
:100d10004f04be000000060003003700b0cf1000f3
:100d2000050032000201e900800178000200e000c5
:100d3000faff3a00000005000300780000000600fa
:100d40008001780002003700b15978000201e90003
:100d50000200e000fcff3a0000000600889fbe0091
:100d60008a1f780000047800c80090006801900095
:100d70000000eb00828f50003c0039001800780022
:100d80002200290002016000e20f5100070032003a
:100d9000012024000000e00001003d0001202000af
:100da000008c70000080eb0030003700020026004d
:100db00002006000820f500009003a0038009000e5
:100dc000808f500006003900080078008d00070071
:100dd000800078000080eb000100e00023003a0072
:100de0001805780000c020000000650018003a00d7
:100df000a80490006002200008004000808f54008a
:100e000013003a00002020001c0307002004980073
:100e10000000e00005003a00290498004904980009
:100e20008904e80039049800080037000a60a0002f
:100e30000a0c7800400498000120200080804000c7
:100e400031049800400c9800500c98000c000700ea
:100e5000280090005004980038009000600498002a
:100e600000002600180c70000000eb004f05780011
:100e70004f04be0000000600207e20009b003700cb
:100e8000881f780068fe20001804e00003003a0084
:100e9000f9ff070020c0b300004c78004f04780031
:100ea00000000600889fbe0000047800080078005b
:100eb000540007008004780000042000180060003f
:100ec0000200320028009000870207000000eb00bb
:100ed00020049800384090000004e0000500350030
:100ee0000000fb00c2fe07000000e000010032002d
:100ef0008084eb00181090000000e0000800320031
:100f000006ff07000000e000010032008084eb00d3
:100f100018109000740207000000eb0010149800f5
:100f20000008200018006000150032000001eb00ee
:100f30006000b800e3ee20000202d00063027a00f5
:100f4000880f520005003a000000400081804800f0
:100f5000008041000008eb000600370061004000ff
:100f6000e08048000201e800e80f5000e08f5800e0
:100f7000f0ff3a00080078005b0207000e0037001f
:100f8000000c780000c0eb003044980060022000a4
:100f90000800400020049800400498005004980085
:100fa000400c980060049800500c98007004980061
:100fb00076004400000c9800090078004f04be0041
:100fc00000000600881f78000004eb006140b800b4
:100fd000e2ff2f00f3ff2f0003050700c2ef200000
:100fe000620078000000e00001003200adff070061
:100ff0000804e800e80f5400f4ff3a004f047800ba
:1010000000000600889fbe00000478000800e00091
:101010000e003a008004eb008800d000e0ee2000d3
:10102000610078000000e00004003200f5ff0700d6
:101030000000e00001003d008084eb000804e800af
:10104000e80f5400f4ff3a002500370000002200aa
:10105000180060008004eb0021003200a80490001a
:101060000f00370009015100384090000000fb00dc
:101070008900780067fe07000000e00007003c00e0
:10108000280090004004980060049800500c9800dc
:101090001890a0008084eb00110037008084440089
:1010a00048019000828f5400eeff39002800900024
:1010b000400498009800780002c02000028160007f
:1010c00001003a003800900001e8a300020032005d
:1010d0006004980001003700500c98008004eb0079
:1010e000090078004f04be00000006000100200047
:1010f0000100e00008003200010080000100e00073
:10110000050032008100e900010088008100d00064
:101110000200800000b1780000000600889fbe0039
:1011200000047800010078008204780088017800cb
:101130000901780011002000a3fe0700890f50006c
:10114000010032000004eb00080078004f04be00ec
:10115000000006000000fa00e88157004fb9970030
:10116000e1e92000e0882000020007000080fa008a
:10117000000006006200fa00889fbe008a1f780007
:10118000000578008104780002047800830078006c
:1011900080f92f000f004000690407009a979f0014
:1011a000a9979f000000eb00b09f9f001885fb00ef
:1011b0008a04fb000a05ea004f55de0050022000b9
:1011c000808f54000d003200e10f55000b003a00f3
:1011d0000a017800880078002f9097009f9197006f
:1011e00003000100a0979f000000e0008e00320085
:1011f0003f9897000000e800b09f9f000a04440059
:1012000050022000808f5400040032000900e000ea
:10121000e6ff3a003f989700840037000000eb009b
:10122000909f9f00809f9f00f0979f00e0979f00f6
:10123000d0979f00c0979f000700370081fd2000d6
:101240000100500000004000c1fc20006100780057
:10125000df98970001007000d09f9f0088047800fd
:1012600009047800384578008a00fb0080fd2000e2
:101270002c0207000000e000f0ff3a00a1c2b3001a
:10128000814f55000e003a00cf8897000180e90099
:10129000c08f9f0010007800c09f9f000000e000fa
:1012a00005003d000000ea00c09f9f005f98970086
:1012b0000020a000d09f9f000904e8000f00370025
:1012c000c09f9f000000eb0005003700f2ff2700e1
:1012d000820f5000020032006a01b9000280400013
:1012e0000904780088047800b900fb000103b1000c
:1012f000e98f5000f5ff3600c09f9f00e0c2b300a9
:10130000984f1000020032000080eb0019003700f7
:10131000a0c2b300d84f100007003a00cf88970052
:101320000180e900c08f9f0010007800a09f9f00ff
:101330000804e800100037000000eb00a09f9f00a9
:101340008800780005003700f3ff2700830f500066
:10135000020032006a02b900040041000104780072
:10136000880078003101fb000203b100e90f510051
:10137000f5ff3600a09f9f00984478008900fb008d
:1013800040fc2000e70107000000e00002003200fe
:101390000804e800010037008044eb00c97f9f008b
:1013a00080c6b30080cf540004003a0098cf1400e8
:1013b0000a003a006640500006003700c0c6b3007d
:1013c00080cf540005003a0098cf140003003a0083
:1013d00065404000c07f9f000804e8001801fb0042
:1013e000e3fb2f008f81410081f92f008f804000a7
:1013f000a0f92f000f004000100007000000e000df
:1014000009003a00e1fb2f008f804000a0f92f0077
:101410000f0040000e0307000000e000020035004e
:101420000804e80061ff37000080eb004f057800fa
:101430004f04be000080fa0000000600889fbe0036
:101440008a1f780000047800e0c6b300804f510086
:10145000c100320015003c006b405000804f51002d
:10146000240032000a003c0070405000804f5100c0
:10147000fa00320065404000804f510068003200a1
:1014800050c2b300804f51000b013a0007013700f2
:1014900040c6b300804f51001b0032006540400041
:1014a000804f510004013a001700370030c7b300e5
:1014b000804f5100e900320007003c0064405000ba
:1014c000804f5100560032000040e800804f51002c
:1014d000f9003a00d300370050c7b300804f5100e5
:1014e0004f00320063404000804f5100f2003a004c
:1014f0004b0037001181e9008208780078009000e5
:1015000012417800ea00370028609000c4c6b3009a
:10151000844f500007003a00110278006400520026
:10152000800878001002be004fabde008603780012
:101530001100370014c7b300844f5000030032007d
:10154000a4c6b300844f500006003a001102780090
:1015500068005200800878003002be002003be0000
:10156000050037001180e90080087800100278003b
:10157000cfa2de00612bb900049cbe000694be0021
:101580002860900081c6b300814f50000d003200ea
:1015900021c6b300814f500004003a000402fb0052
:1015a000cfa2de00612bb9000800370041c7b300ad
:1015b000814f500003003200e6c04000814f5000d0
:1015c00004003a00cfa2de00612bb900049cbe00eb
:1015d0000694be003802be002803be0078009000ca
:1015e000d1c2b300e00f5200e08f5a00e00f5b0061
:1015f000e08f5b0008003500881090000118a30000
:1016000002003200b1c2b300030037000108a3009a
:101610004c00320001c2b3008171780047003700ee
:1016200028609000c4c6b300844f500006003a0002
:101630001102780064005200800878001002be0099
:101640006033b8001100370014c7b300844f500056
:1016500003003200a4c6b300844f500006003a00d5
:101660001102780068005200800878003002be0045
:101670002003be00050037001180e90080087800d3
:10168000100278008002eb006033b800049cbe00ba
:101690000694be002860900081c6b300814f5000c0
:1016a0000d00320021c6b300814f500004003a0003
:1016b0000482fb008002eb006033b80008003700b2
:1016c00041c7b300814f500003003200e6c0400024
:1016d000814f500004003a008002eb006033b800f4
:1016e000049cbe000694be00081090000038a300c1
:1016f000140032003802be002803be00e00f520082
:10170000e08f5a00e00f5b00e08f5b000d003200bd
:1017100080c7b300804f51000300320080c5b30082
:10172000804f510007003a007800900001c3b300d9
:10173000817178000000e800827178000000e80004
:101740007004980078009000808141006304980044
:10175000824078003e00370028619000c3c6b30085
:101760001180e900834f5100220032000a003c0042
:10177000e4c15100834f51002500320083c1e800cd
:10178000834f510013003200e8c15100834f5100d4
:101790001e003a000a00370043c7b300834f5100d0
:1017a0001b003200e6c14100834f51001800320097
:1017b000e9c15100834f510014003a000500370081
:1017c0008008780010007800485c90000848780095
:1017d000410037008008780010007800680a900007
:1017e000cfa2de00612bb9000498be000690be00b7
:1017f00039003700800878001000780068099000f0
:10180000cf91de000288be00330037001180e9006e
:101810008008780010007800680c900008087800b4
:101820002d0037001180e900800878001002780050
:10183000cfa2de00612bb900049cbe000694be005e
:1018400078009000808141006304980081c7b30054
:1018500008007800cf0007001f0037001180e90062
:1018600080087800100578006a049800d80c900071
:101870000900e00004003d000a007800b500070000
:101880008004780007003700090178008000eb0031
:101890000a00780020fd07000000e000010032008f
:1018a0008a045000190c98000b0037007800900053
:1018b0008271780006003700780090008081410036
:1018c0000204e00001003a0052c2b30082497800ed
:1018d0000000e800700498000000eb004f0578005d
:1018e0004f04be00000006000000e0002f003200a0
:1018f000c0017800e38f51002c0036000308a300dc
:101900002a003a00217f80000100e000020032003e
:10191000810f50000400310011009800207f8800e2
:101920001600370082007800110190000200e000ec
:1019300002003200800f5100faff390011027800d6
:1019400084824000850f500018003900808f5200bb
:1019500003003a00830842000100780007003700c6
:101960000200e0000300320083014000830f5100b9
:101970000e0039001200980090009800900090002e
:101980000100e0000900320010014000828f500089
:1019900006003a0022fe20000009eb00100178004a
:1019a000110841009100900011009800000006000d
:1019b000889fbe0000047800117f80000100e000d5
:1019c00002003200010078000d003700217f800006
:1019d00040fe200004003700910f5400250036001f
:1019e0000180e800910090000100e000faff3a0059
:1019f00010003700920f54001e0036000280e800ed
:101a0000100178000200e000faff3a0011017800ae
:101a1000217f800040fe200004003700910f540019
:101a2000140036000180e80091009000828f500081
:101a3000faff3a00497f8000888f5400010031008e
:101a40008804780009007800480007000000e000e2
:101a500004003a00888f5400050032008904d10048
:101a6000f5ff3700091878009fff0700d2ff370005
:101a70000000eb004f04be0000000600881f780045
:101a8000630440000800a1008000eb00800f5400b8
:101a900021003600e30f540001003e004800200002
:101aa00008007800c2ff07008000eb000000e000a3
:101ab0001900320090007800910178006481510093
:101ac000880f5100030031001101900002087800d6
:101ad000070037000881400002087800910190005b
:101ae000130198001001780011091400880878008b
:101af000100178000000eb000200e000040032005a
:101b0000920190000300e000010032000280e80032
:101b1000107f88008180e800010078004f04780081
:101b200000000600020037000304e0000600320057
:101b30000001780002007800b041780081cf5100a8
:101b4000f9ff3a00010037000001eb0002007800c5
:101b50000000060080007800010178003104e000f8
:101b6000fdff3a00000051000000060080007800f0
:101b70000000eb000100e0000500340001007800e7
:101b8000effb0700e10f400001003a000000eb000e
:101b900000000600fc874700889fbe008a9fbe00a9
:101ba0008c9fbe008e1f78000006780080c5b300b1
:101bb00080cf50000a0032007740400080cf5000b4
:101bc0000a0032006940400080cf50000b00320014
:101bd00050f9200080bf9f00ae0020000a003700af
:101be00042f8200082bf9f000600370053f9200012
:101bf00083bf9f008e0020000300370054f92000af
:101c000084bf9f000e0120003c02be002c03be00da
:101c10000605be000404be0040c6b30080cf5000dd
:101c2000030032006540400080cf50000b003a00b6
:101c3000e00f5200e08f5a00e00f5b00e08f5b0086
:101c400006003d006000b8006011b80004045000b8
:101c5000858458000605590087855900e80f57000c
:101c60000400320040002000f00f570038003a0016
:101c70000100370030002000e00f5400e08f5c00ce
:101c8000e00f5d00e08f5d0004003a00dc0890008a
:101c90008d0120000100e000060032008e00e90006
:101ca000888060008fba9700e5c07800f1ef9f0050
:101cb0007d012000800078008100e90005003300ec
:101cc0008b05d1000a85d3008984d3000884d30012
:101cd000f9ff3700089ebe000a96be0012003700ca
:101ce0008d06e9008e00e900848060000fb997003e
:101cf000e2c1780082fd2f000f01410003f17e0058
:101d0000800078008100e900050033008783d1005e
:101d10000683d3008582d3000482d300f9ff370005
:101d2000049ebe000696be003c02be002c03be0010
:101d3000e00f5200e08f5a00e00f5b00e08f5b0085
:101d40008b0034000d00e000e5ff3c008800370008
:101d50002c60900081c6b300814f50000b00320010
:101d600006003c000004e00008003200e6c050001d
:101d7000814f50004e003a0004003700c1c6b30046
:101d8000814f50004a003a00210037000800e0006f
:101d900004003a005c0890008d0120000000e00083
:101da00006003200110009000e84d8000fb9970018
:101db000e2c07800f1ef9f007d01200011000900d2
:101dc0000e84d8000a003700110009000e04d80064
:101dd0008d06e9000e81b900020454008fb8970007
:101de00061417c0081fd2f008f80400082f07e00e9
:101df000000478000800e000020032000d00e0005e
:101e0000f1ff3c00cfc4de00614db9002500370072
:101e1000e00f5400e08f5c0004003a005c08900082
:101e20008d0120000000e000070032006171b90060
:101e30000800be00690107008fb99700e3417800f0
:101e4000f3ef9f007d0120006171b9000800be0022
:101e5000520107000b0037006171b9000800be0095
:101e60003f0107008d06e90000f1b90002045400ab
:101e70000fba9700e4427c0084fd2f000f0242005d
:101e800005f27e000004be00e00f5000e08f580015
:101e9000020032000d00e000efff3c004fcdde00fd
:101ea0008a057800089ebe000a96be003000370002
:101eb000e00f5400e08f5c00e00f5d00e08f5d00fc
:101ec00004003a005c0890008d0120000000e00052
:101ed000090032006172b900612bb9000800be0030
:101ee0000a01be00e60107000fba970064427800bd
:101ef000f4ef9f007d0120006172b900612bb900f1
:101f00000800be000a01be00d60107000d00370020
:101f10006172b900612bb9000800be000a01be0061
:101f2000db0107008d06e90000f2b900040454004b
:101f30008fba970065427c0085fd2f008f8242009a
:101f400084f27e00009ebe000296be003c04be00ed
:101f50002c05be00e00f5400e08f5c00e00f5d0038
:101f6000e08f5d00020034000d00e000e8ff3c005f
:101f7000e80f570010003a000c1090000038a30042
:101f80000d003200f78f560006003e0085fd2f0041
:101f90008f824200e5c07e0000c3b30080cf5000b6
:101fa000050032008d06e90002c3b30081fd2f0059
:101fb0008f80400082f07e0078811600120e98001b
:101fc0006c00900083fd2f008f8141008d804100c7
:101fd0005bfb07001c089000dc089000810f50009c
:101fe00006003d0000805000000e98000c1090008c
:101ff0000040a100001698000f0037000100e0002b
:102000000d003d008c109000f4806000f08f5000b7
:1020100009003a007c099000fc009000810051000a
:102020000c09900082805000008050004240a900be
:1020300001003400000e98004f0778004f06be00e4
:102040004f05be004f04be00cf01b10000000600e6
:102050000400fa00889fbe008a9fbe008c1f780093
:102060000004780001067800f80d900078009000d8
:10207000808555000808900080855500180890005c
:10208000808555002808900080855500380890000c
:102090008085550048089000808555000002220088
:1020a00090bf9f0000032300a0bf9f000810900076
:1020b0000028a30015003a000b00e00013003400d4
:1020c0000b0578008a047800e20f55000100360005
:1020d00029002000c801900009017800ee80570017
:1020e0005800900003000100500498000000e00038
:1020f0008c0032006808900009004000600c9800d5
:10210000090555004240a900eeff3c00780190000f
:102110000200e0000c003400c80190008c00780040
:102120005800900003000100500498008080eb00ec
:102130000000e0007c003200e80890007800900089
:1021400000804000600c9800880c90000900e000be
:102150001100340009057800e28f540001003600b8
:102160002a002000c80190000a017800ec80570086
:102170005800900003000100500498000000e000a7
:1021800068003200680890000a004000600c980067
:102190008a845400edff3700180990000200e00027
:1021a0000c003400c8019000e80090005800900036
:1021b00003000100500498008080eb000000e00064
:1021c00059003200e8089000180890000080400094
:1021d000600c9800a80c90000900e0001100340089
:1021e00009057800e28f5400010036002a00200023
:1021f000c80190000a017800ec8057005800900058
:1022000003000100500498000000e0004500320087
:10221000680890000a004000600c98008a8454000e
:10222000edff3700380990000200e0000e00340096
:10223000e80090001808900080804000c8019000dd
:102240005800900003000100500498008080eb00cb
:102250000000e00034003200e808900038089000e8
:1022600000804000600c9800c80c90000900e0005d
:102270001100340009057800e28f54000100360097
:102280002a002000c80190000a017800ec80570065
:102290005800900003000100500498000000e00086
:1022a00020003200680890000a004000600c98008e
:1022b0008a845400edff3700081090008000eb0086
:1022c0000028a300180032000b00e00016003400c4
:1022d0008b04780009057800e28f54000100360075
:1022e0002a002000c80190000a017800ee80570003
:1022f0005800900003000100500498000000e00026
:1023000008003200680890000a004000600c980045
:102310008a8454004240a900eeff3c008000eb009c
:10232000010037008080eb00010078004f06780044
:102330004f05be004f04be000080fa0000000600fa
:10234000010878000000060000c0da000000060066
:1023500000c0da000000060000c0da00000006003d
:10236000839f68000100e00002003d006000100053
:10237000e08018000300e00002003d006001110051
:10238000e0811900050007004f00e00002003b005b
:1023900060001000e0801800000006006022b80015
:1023a000060220000000d0008180d2000482d2000a
:1023b0008582d2000000a0000202520083825a00ef
:1023c000030031000202420083824a000000a100a3
:1023d0000603e900f3ff3a0000000600efff0700e4
:1023e0000400be0000000600020ab900001bb9008c
:1023f0000200b80081004200810043000000060096
:10240000889fbe008a9fbe0030044200b0844a000c
:1024100030054b0090854b006000b1000898be006d
:102420000a90be000440e10005c8e10006d0e100ca
:1024300007d8e10002003100680040001008e80001
:102440004f05be004f04be0000000600889fbe007e
:102450008a9fbe003004be002005be000418540050
:1024600005985c0006185d0007985d0011002000cb
:102470000440e10005c8e10006d0e10007d8e10012
:10248000010039008000eb00108810004f05be00ed
:102490004f04be00000006001200fa00889fbe0034
:1024a0008a9fbe008c9fbe00e0b79f00f1b79f00df
:1024b00082bf9f0093bf9f000605be000404be00bc
:1024c0000000eb00d0b79f00c0b79f00b0b79f00df
:1024d000a0b79f0090b79f000006eb005fb1970088
:1024e000cfb09700820141003fb097000200e000aa
:1024f00004003d00370007007e805700c0ff070042
:1025000003003700330007007e805700cfff07002d
:10251000dfb697000d00e0000c0035006fb29700a9
:10252000ffb297000fbb97009fbb970010002000e1
:10253000010020006011b800000272008182720068
:1025400002037300838373001b0007000c06e8007e
:1025500001042000810f5600e0ff3a000d00e0006a
:1025600004003d000802be000a03be007e80570042
:10257000a3ff07005fa897000000e00005003a00f5
:102580001fb29700afb297003fb39700cfb3970049
:10259000090007006fb09700ffb097000fb99700d0
:1025a0009fb997004f06be004f05be004f04be0006
:1025b0000080fa000000060001000700000006008d
:1025c000a4b79f00b5b79f00c6b79f00d7b79f00bd
:1025d000000006004f09de0082817100b3b79f0042
:1025e0004f01de008180400082807000a1b79f0013
:1025f0008fb097004f09de0000004000020070001d
:1026000090b79f007fa897004f01de0081804000b7
:102610008280700081b79f000d0007004f3ade00f6
:102620000000400004007000f0af9f0008000700a9
:102630000402420085824a0006034b0087834b0058
:10264000dfff07000802be000a03be00000006000c
:102650002fb29700bfb297004fb39700dfb3970038
:1026600000000600881f780018002000881f7800ee
:1026700089ff07008f87e9004f04780000000600fb
:10268000801feb0084ff07008f87e9000000060031
:10269000889fbe008a9fbe00e00f5000e08f580068
:1026a000e00f5900e08f59000c003d006044b80075
:1026b0006055b8000000540081805c0002015d009c
:1026c00083815d00180020001500070008003d0010
:1026d000180007000004eb00050037000004eb00c1
:1026e0000f00070002003d00120007001800200044
:1026f000dcff07000800e000060032006022b8009e
:102700006033b8000000520081805a0002015b0073
:1027100083815b004f05be004f04be000000060031
:10272000e00f5200e08f5a00e00f5b00e08f5b008b
:10273000000006006044b8006055b8000402540070
:1027400085825c0006035d0087835d000000060053
:10275000889fbe008a9fbe008c1f7800e00f50004b
:10276000e08f5800e00f5900e08f59000d003d0048
:102770006044b8006055b8000000540081805c00df
:1027800002015d0083815d001c0020000820e10043
:1027900009a8e1000ab0e1000bb8e1000d003d001e
:1027a000080037000006eb00e00f5200e08f5a00ef
:1027b000e00f5b00e08f5b0006003d006044b80066
:1027c0006055b8000402540085825c0006035d0079
:1027d00087835d00aaff07000c00e00006003200be
:1027e0006022b8006033b8000000520081805a00b7
:1027f00002015b0083815b004f0678004f05be003d
:082800004f04be0000000600b9
:020000040000fa
:10280800313100003a350000333a00003534000019
:1028180000410000707200002020000034200000f9
:102828003230000032310000003000002e3200004b
:10283800000d00000a48000050480000494c000004
:102848004b42000044200000257300002053000084
:102858007461000072740000696e0000672e000049
:10286800202500007320000025730000000d0000e3
:102878000a5000004f520000544200003a20000065
:1028880025580000000d00000a4c0000616e000091
:10289800677500006167000065200000636f000035
:1028a80064650000206900007320000025580000be
:1028b80000200000736500006e64000020640000c2
:1028c8006576000069630000652000004944000047
:1028d800202500005820000000200000483a000091
:1028e8002025000058200000000d00000a420000ca
:1028f80020310000206400006e0000000d0a000076
:10290800422000003120000075700000000d00001a
:102918000a42000020320000206400006e0000001f
:102928000d0a0000422000003220000075700000ef
:10293800002000004861000072640000207200005e
:1029480065730000657400000049000046430000fc
:102958000045000050540000004500004c420000b3
:1029680000490000444400000044000053520000a5
:10297800005000005354000000520000524700006d
:102988000057000052470000004100004346000085
:1029980030000000414300004631000000410000c3
:1029a8004346000032000000414300004633000067
:1029b800004100004346000034000000414300008d
:1029c8004635000000410000434600003600000084
:1029d8004143000046370000005000004f4c000003
:1029e80030000000504f00004c3100000050000043
:1029f8004f4c000032000000504f00004c330000e4
:102a0800005000004f4c000034000000504f000000
:102a18004c350000005000004f4c0000370000000b
:102a2800504f00004c380000005000004f4c000090
:102a380039000000504f00004c61000000500000b9
:102a48004f4c000062000000504f00004c63000033
:102a5800005000004f4c000064000000504f000080
:102a68004c650000005000004f4c0000660000005c
:102a7800525000004c30000000520000504c000042
:102a880031000000525000004c320000005200009b
:102a9800504c000033000000525000004c3400003d
:102aa80000520000504c0000350000005250000059
:102ab8004c36000000520000504c00003700000067
:102ac800525000004c38000000520000504c0000ea
:102ad80039000000525000004c6100000052000014
:102ae800504c000062000000525000004c6300008f
:102af80000520000504c00006400000052500000da
:102b08004c65000000520000504c000066000000b8
:102b1800524e00004d0000005253000054000000c7
:102b280045580000440000005253000043000000d4
:102b3800303300003400000030330000350000005e
:102b4800303300003600000030330000370000004a
:102b58003033000038000000303300003900000036
:102b680030330000610000003033000062000000d4
:102b78003033000063000000444b000041000000b7
:102b8800454b000031000000454b000032000000ba
:102b98005052000031000000505200003200000086
:102ba8005052000033000000505200003400000072
:102bb800505200003500000050520000360000005e
:102bc8005052000037000000505200004d00000035
:102bd800414b000031000000414b00003200000072
:102be800414b000033000000414b0000340000005e
:102bf800414b000035000000414b0000360000004a
:102c0800414300004b000000303500003000000058
:102c1800303500003100000030350000320000007f
:102c2800303500003300000030350000340000006b
:102c38003035000035000000303500003600000057
:102c48003035000037000000303500003800000043
:102c58003035000039000000303500006100000008
:102c680030350000620000003035000063000000cd
:102c780030350000640000003035000065000000b9
:102c880030350000660000003036000030000000db
:102c980030360000310000003036000032000000fd
:102ca80030360000330000003036000034000000e9
:102cb80030360000350000003036000036000000d5
:102cc80030360000370000003036000038000000c1
:102cd8003036000039000000303600006100000086
:102ce800303600006200000030360000630000004b
:102cf8003036000064000000303600006500000037
:102d08003036000066000000303700003000000058
:102d1800303700003100000030370000320000007a
:102d28003037000033000000303700003400000066
:102d38003037000035000000303700003600000052
:102d4800303700003700000030370000380000003e
:102d58003037000039000000303700006100000003
:102d680030370000620000003037000063000000c8
:102d780030370000640000003037000065000000b4
:102d880030370000660000003038000030000000d6
:102d980030380000310000003038000032000000f8
:102da80030380000330000003038000034000000e4
:102db80030380000350000003038000036000000d0
:102dc80030380000380000003038000039000000ba
:102dd8003038000061000000303800006200000058
:102de8003038000063000000303800006400000044
:102df8003038000065000000303800006600000030
:102e08003039000030000000303900003100000087
:102e18003039000032000000303900003300000073
:102e2800303900003400000030390000350000005f
:102e3800303900003600000030380000370000004c
:102e48003039000038000000303900003900000037
:102e580030390000610000003039000062000000d5
:102e68003039000063000000306100006400000099
:102e780030390000650000003039000066000000ad
:102e880030610000300000003061000031000000b7
:102e980030610000320000003061000033000000a3
:102ea800306100003400000030610000350000008f
:102eb800306100003600000030610000370000007b
:102ec8003061000038000000306100003900000067
:102ed8003061000061000000306100006200000005
:102ee80030610000630000003062000064000000f0
:102ef80030610000650000003061000066000000dd
:102f08003062000030000000306200003100000034
:102f18003062000032000000306200003300000020
:102f2800306200003400000030620000350000000c
:102f380030620000360000003062000037000000f8
:102f480030620000380000003062000039000000e4
:102f58003062000061000000306200006200000082
:102f6800306200006300000030620000650000006d
:102f7800306200006600000030630000300000008e
:102f880030630000310000003063000032000000b0
:102f9800306300003300000030630000340000009c
:102fa8003063000035000000306300003600000088
:102fb8003063000037000000306300003800000074
:102fc8003063000039000000306300006100000039
:102fd80030630000620000003063000063000000fe
:102fe80030630000640000003063000065000000ea
:102ff800306300006600000030640000300000000c
:10300800306400003100000030640000320000002d
:103018003064000033000000306400003400000019
:103028003064000035000000306400003600000005
:1030380030640000370000003064000038000000f1
:1030480030640000390000003064000061000000b6
:10305800306400006200000030640000630000007b
:103068003064000064000000306400006500000067
:103078003064000066000000306500003000000089
:1030880030650000310000003065000032000000ab
:103098003065000033000000306500003400000097
:1030a8003065000035000000306500003600000083
:1030b800306500003700000030650000380000006f
:1030c8003065000039000000306500006100000034
:1030d80030650000620000003065000063000000f9
:1030e80030650000640000003065000065000000e5
:1030f8003065000066000000304600003000000027
:103108003046000031000000304600003200000068
:103118003046000033000000304600003400000054
:103128003046000035000000304600003600000040
:10313800306600003700000030460000380000000c
:103148003046000039000000524900004f000000de
:10315800534800005200000054450000520000008f
:1031680043410000450000004448000052000000b0
:1031780030660000660000000d0a000020500000c4
:1031880061750000736500002f6200007265000021
:10319800616b000000200000636f000064650000a0
:1031a800322000006f6e000000200000636f0000f6
:1031b80064650000322000006f66000066000000b1
:1031c8000d0a0000503a0000202500003458000085
:1031d800204300003a20000025320000582000005b
:1031e800000d00000a4d00002025000030320000cc
:1031f800582000002530000032580000202500002b
:10320800303200005820000020000000202d00006f
:10321800204900006e760000616c000069640000bf
:1032280020730000746100007475000073200000b2
:103238002d0000002020000025330000642000003d
:103248002025000033640000000000000e0000008c
:103258007e000000160000007c0000001e00000038
:103268007a00000026000000780000002500000019
:10327800760000002e0000007400000036000000f8
:10328800720000003d000000700000003e000000d9
:10329800b000000046000000b20000004500000039
:1032a800b40000004e000000b60000005500000009
:1032b800b800000066000000ba0000000d00000021
:1032c8006e000000150000006c0000001d000000ea
:1032d8006a00000024000000680000002d000000c3
:1032e800660000002c0000006400000035000000ab
:1032f800620000003c000000600000004300000085
:10330800c000000044000000c20000004d000000a2
:10331800c400000054000000c60000005b0000006c
:10332800c8000000580000005e0000001c000000fb
:103338005a3800001b00000058000000230000005d
:10334800560000002b00000054000000340000006c
:103358005200000033000000500000003b00000055
:10336800d000000042000000d20000004b00000026
:10337800d40000004c000000d600000052000000fd
:10338800d80000005a000000da0000001200000017
:103398000a00000011000000070000001a000000e9
:1033a8003800000022000000360000002100000064
:1033b800340000002a000000320000003200000043
:1033c8003000000031000000f00000003a0000006a
:1033d800e000000041000000e20000004900000099
:1033e800e40000004a000000e60000005900000068
:1033f80008000000140000000c0000002900000074
:10340800f2000000140000000c000000670000003b
:10341800cc00000064000000ce0000006b0000003b
:10342800f800000075000000fc00000072000000b9
:10343800fa00000074000000fe0000006c000000ac
:10344800dc0000006b0000001000000069000000b4
:103458002000000077000000a000000075000000b8
:103468001200000073000000140000007200000049
:1034780024000000700000002c0000007e00000006
:103488000c0000007d000000160000007400000021
:10349800180000007a0000002800000071000000f9
:1034a800ce000000840000002e000000790000001b
:1034b8001e000000760000003e000000050000002d
:1034c80098000000060000009600000004000000bc
:1034d800940000000c0000009200000003000000af
:1034e800a20000000b000000a40000008300000000
:1034f800a60000000a000000a8000000e10000008b
:103508009c000000010000004a9e00000900000025
:1035180042ae00007800000046ac00000700000042
:103528004e0000005d000000ca0000006be00000d3
:10353800f800000074e00000fe00000075e00000e4
:10354800fc00000072e00000fa00000070e00000db
:10355800ccbc000071e00000cebe00006ce00000b2
:10356800dc00000069e00000ea0000007de00000e7
:10357800de0000007ae00000ee0000005ae00000e3
:10358800da00000014e100000e0000007ce00000fa
:10359800900000000d0a0000553a000020200000ad
:1035a8002530000032580000000d00000a550000c8
:1035b800523a000020250000303200005820000058
:1035c800002000005374000061740000757300004f
:1035d8003a20000025580000202d00003e20000061
:1035e80025580000000d00000a4c00002063000070
:1035f800747200006c20000063680000616e0000b7
:103608006765000064200000746f00003a20000025
:10361800256400002000000070720000657300003f
:1036280073000000726500006c65000061730000a3
:10363800650000000d0a00004c20000073680000bf
:10364800696600007420000063680000616e000075
:103658006765000064200000746f00003a200000d5
:1036680025640000200000000d0a00004c20000026
:10367800616c00007420000063680000616e000047
:103688006765000064200000746f00003a200000a5
:103698002564000020000000206300006f64000023
:1036a80065320000206f00006e200000002000003e
:1036b800636f000064650000322000006f66000040
:1036c8006620000000000000045a00006c0500009d
:1036d800300000000634000000070000560000001b
:1036e8000868000000090000540000000a520000a9
:1036f800000b0000500000000cc00000000d00008e
:10370800d00000000ed20000000f0000d40000001e
:1037180010e0000000110000f000000012c20000dc
:1037280000130000c4000000146c00000015000025
:103738006600000016580000001700006400000032
:103748001860000000190000320000001a6a00002a
:10375800001b0000360000001c620000001d000075
:10376800380000001e7c0000001f00007a000000e6
:10377800207800000021000076000000227400007c
:1037880000230000720000002470000000250000e3
:10379800b000000026b2000000270000b4000000be
:1037a8002db60000002e0000b80000002fc8000051
:1037b80000300000c600000031ca000000320000de
:1037c8007e00000033d6000000340000d80000005e
:1037d800357e000000360000e200000037e40000fb
:1037e80000380000e60000002cf20000003900005c
:1037f8005e000000e10a000000e20000070000008f
:10380800e508000000e000000c0000004cce0000bd
:10381800be280000da00000049cc0000bc2a0000e5
:10382800babe00004ffe000000500000f800000083
:1038380052fc000000510000fa0000004adc0000c1
:10384800004d0000ea0000002b4c0000004b000077
:10385800de0000004eee00000059000020000000cd
:103868005a240000005b0000280000005c100000e3
:10387800005d0000140000005e180000005f0000fa
:103888001a0000006012000000610000160000002d
:10389800622c00000063000048000000479c000004
:1038a800005700001e000000562e000000580000bf
:1038b800da000000293e0000004800000e00000069
:1038c8004690000000530000a000000054220000b1
:1038d80000550000260000003a980000003b000058
:1038e800960000003c940000003d0000920000009b
:1038f8003ea20000003f0000a400000040a6000017
:1039080000410000a8000000424a0000ac4300004b
:1039180042ae0000444600009e4500004e000000f4
:10392800313100003a350000333a000035340000e8
:1039380000410000707200002020000034200000c8
:103948003230000032310000000d00000a4800004b
:1039580050480000494c00004b420000442d000034
:1039680050530000322000004d6f000075730000b6
:103978006520000053740000617200007469000043
:103988006e6700002e20000025730000202500002f
:10399800730000000d0a00002564000020250000c7
:1039a800580000000d0a00004e6f0000206d000056
:1039b8006f750000736500002070000072650000dc
:1039c800736500006e740000000d00000a200000fe
:1039d8002558000000000000313100003a35000091
:1039e800333a0000353300000041000070720000d7
:1039f8002020000034200000323000003231000066
:103a0800000d00000a48000050480000494c000022
:103a18004b420000442d00005053000032200000ab
:103a28005374000061720000746900006e67000042
:103a38002e200000257300002025000073000000e0
:020000040000fa
:103a48003a68ef002ca3ef00c9e2a900c9c2a90097
:103a5800c9a2a800c8a2a900c8e2a800cf02a9006c
:103a68008400a90070002000a420b7008200a800ec
:103a78009400a8009021ef009221ef0003c02100dc
:103a8800030078009021b70082ff2f00810c80008e
:103a9800010061003000b300800c8800f0012000b4
:103aa8009221b70092a1a800010a2000a10c880069
:103ab8009621ef0084c0a90094c0a80004702000db
:103ac80004007800a620b7009a21ef009c21ef009f
:103ad800030078009a21b700a0192000100861009f
:103ae800f00120009c21b7009ca1a800f10c8800df
:103af800a021ef0084c0a90094c0a90004007800a8
:103b0800a620b7009560a9009580a900103a80000a
:103b1800f00bb2007205200061042000237420001d
:103b2800814978008249780080497800f00f2e009a
:103b3800d406b6000030b300a0368800d0a2a90091
:103b480010022000401188002062a80021e2a8008d
:103b58002342a80040402900801f7800d040290057
:103b6800801f780090412900801f7800d0412900eb
:103b7800801f780075f50700f0002000c822b70004
:103b8800d002a800501680006f006000d042880064
:103b9800e8875700d202ab000200320070004000f4
:103ba800d0428800ca02f800b0432900801f78007c
:103bb80066f507005a08f80070442900801f78004d
:103bc80062f50700e8875700000006000200fa00c7
:103bd800889fbe008a9fbe008c1f78000044780032
:103be800e54f51002d0432000f003600f04f510010
:103bf800ba00320056003e00e84f51000500390077
:103c0800674061002ee8b7005cc8bf00e14f500074
:103c18007f0532004f0678004f05be004f04be00f6
:103c28000080fa0000000600e14f5100cf03320087
:103c380057003100830020000804e00001003a002a
:103c48008001eb008180fb000041eb000108a3002c
:103c58000100320042c0b300024078000014a00006
:103c68000118a300010032000041780002407800ea
:103c78000004a0000128a3000100320000417800e0
:103c88000280fb00030070009440ab00feff3a0086
:103c980000004000a041880000002c003428b70034
:103ca800a04180008080d100808068004281de00d1
:103cb800810069004381de00810069004481de00e3
:103cc800810069004581de00810069004681de00cf
:103cd800810069004781de00810069004881de00bb
:103ce800810069004981de00810069004a81de00a7
:103cf800810069004b81de00810069004c81de0093
:103d0800810069004d81de004e80de0061006000a8
:103d180081006900e1806000810f500001003a00d5
:103d280035a8a80000012000904188009801e20011
:103d3800feff3a009440a8004f0678004f05be00e9
:103d48004f04be000080fa0000000600b6ff3700ee
:103d5800e24f4100afff3a00d0492900801f7800a8
:103d6800faf4070010c0b3005ce8b7002868ef0059
:103d7800b30d07008f87e9004f0678004f05be0096
:103d88004f04be000080fa0000000600a6ff3700be
:103d9800e24f510029033200e34f51009dff3a00e2
:103da8008184fb00e2822000124178000200fb00bf
:103db800808f5400490632005cc8bf00e2cf500033
:103dc8002b0432000004e00092ff32008200200041
:103dd8000804e00001003a000001eb008040eb001d
:103de8000908a3000100320041c0b3000140780077
:103df8000014a0000918a3000100320080407800d8
:103e0800014078000004a0000928a3000100320046
:103e1800804078008180fb0000c020000100700015
:103e2800000071009440ab00feff3a000000400023
:103e3800a041880000002c003428b700a041800071
:103e48008080d100808068004281de0081006900a6
:103e58004381de00810069004481de008100690041
:103e68004581de00810069004681de00810069002d
:103e78004781de00810069004881de008100690019
:103e88004981de00810069004a81de008100690005
:103e98004b81de00810069004c81de0081006900f1
:103ea8004d81de004e80de00610060008100690007
:103eb800e1806000810f500001003a0035a8a80099
:103ec80000012000904188009801e20099ff32002b
:103ed8009801e200fcff3a0096ff37002c28ec001e
:103ee800404b80000000e000030032005cc8bf00c7
:103ef800e14f5000d60132002a48e2008901320021
:103f0800404b80000000e00086013a005c48e20077
:103f180084013200e241800082027800f34180008f
:103f2800030278000280690063006000990632008d
:103f38002e48ec000080fb00e10460000043eb0029
:103f48000100320046c0b300064578000a14a000fc
:103f58008083d1000708a30001003a0006457800d5
:103f68008a4578000b04a0004283de000608a300ff
:103f7800010032000b4578000a85fb000042200052
:103f88000a0070009440ab00feff3a0000004000b9
:103f9800a041880000002c003428b700a041800010
:103fa8000085d10000056d00c285de000a856d0020
:103fb800c385de000a856d00c485de000a856d00b4
:103fc800c585de000a856d00c685de000a856d00a0
:103fd800c785de000a856d00c885de000a856d008c
:103fe800c985de000a856d00ca85de000a856d0078
:103ff800cb85de000a856d00cc85de008a856d00e4
:104008004d86de004e80de00610560000b006e000c
:1040180061006000800f550001003a0035a8a80033
:1040280000012000904188009801e200feff3a005c
:104038009440a8000040eb000900e00001003200b5
:1040480040c0b300804478000914a0000708a3000a
:104058000100320009407800804378000704a0007e
:104068000608a30001003200074078000083fb0027
:10407800e04080000080fb008043eb000008a300c4
:104088000100320007c8b300874478000964a00023
:104098000018a300010032008943780087447800a3
:1040a8000954a0000028a3000100320089437800c9
:1040b800874478000944a0000038a30001003200ba
:1040c80089437800874478000934a0000048a30099
:1040d8000100320089437800874478000924a00051
:1040e8000058a30001003200894378008744780013
:1040f8000914a0000068a300010032008943780079
:10410800874478000904a0004700de00010032005f
:10411800894378000780fb004400dd00000073003d
:104128009440ab00feff3a0000004000a041880028
:1041380000002c003428b700a04180008083d10003
:1041480080836b00c284de0087836c00c384de003a
:1041580087836c00c484de0087836c00c584de001e
:1041680087836c00c684de0087836c00c784de000a
:1041780087836c00c884de0087836c00c984de00f6
:1041880087836c00ca84de0087836c00cb84de00e2
:1041980087836c00cc84de0087846c004d85de004c
:1041a8004e80de00e103600009006d0061006000e0
:1041b800808f530001003a0035a8a80000012000b4
:1041c800904188009801e200feff3a009440a80060
:1041d800f04080000080fb008043eb000008a30053
:1041e8000100320007c8b300874478000964a000c2
:1041f8000018a30001003200894378008744780042
:104208000954a0000028a300010032008943780067
:10421800874478000944a0000038a3000100320058
:1042280089437800874478000934a0000048a30037
:104238000100320089437800874478000924a000ef
:104248000058a300010032008943780087447800b1
:104258000914a0000068a300010032008943780017
:10426800874478000904a0004700de0001003200fe
:10427800894378000780fb004400dd0006007000d9
:104288009440ab00feff3a0000004000a0418800c7
:1042980000002c003428b700a04180008083d100a2
:1042a80080836b00c284de0087836c00c384de00d9
:1042b80087836c00c484de0087836c00c584de00bd
:1042c80087836c00c684de0087836c00c784de00a9
:1042d80087836c00c884de0087836c00c984de0095
:1042e80087836c00ca84de0087836c00cb84de0081
:1042f80087836c00cc84de0087846c004d85de00eb
:104308004e80de00e103600009006d00610060007e
:10431800808f530001003a0035a8a8000001200052
:10432800904188009801e200feff3a009440a800fe
:10433800390020000218a300da0532000318a30090
:10434800ab0432000508a3005f0432000408a30090
:104358001404320070c04400840020000804e00007
:1043680001003a000002eb000181fb008041eb00f4
:104378000208a3000100320043c0b3008342780062
:104388000514a0000218a30001003200854178003e
:10439800834278000504a0000228a300010032002f
:1043a800854178000080fb000041eb000008a30075
:1043b8000100320002c8b300824278000564a00000
:1043c8000018a300010032000541780082427800fd
:1043d8000554a0000028a300010032000541780020
:1043e800824278000544a0000038a3000100320092
:1043f80005417800824278000534a0000048a300f7
:104408000100320005417800824278000524a000ae
:104418000058a3000100320005417800824278006c
:104428000514a0000068a3000100320005417800cf
:10443800824278000504a0004700de000100320037
:10444800054178000281fb004411dd000380fb0078
:1044580002007000000072009440ab00feff3a00ba
:1044680000004000a041880000002c003428b7005c
:10447800a04180000081d10000016900c281de00f6
:1044880002816900c381de0002816900c481de0007
:1044980002816900c581de0002816900c681de00f3
:1044a80002816900c781de0002816900c881de00df
:1044b80002816900c981de0002816900ca81de00cb
:1044c80002816900cb81de0002816900cc81de00b7
:1044d800828169004d82de004e80de00610160004d
:1044e80003006a0061006000800f510001003a007b
:1044f80035a8a80000012000904188009801e2003a
:10450800feff3a009440a8002a68ef00c28320000a
:1045180012417800e3832000824978001c28ef00cc
:104528001e28ef002848e200bafd3a002a48e200b7
:10453800b8fd3a005cc8bf00e14f5000b5fd3a0035
:10454800800020000804e00001003a000000eb00b1
:104558008180fb000041eb000108a300010032004c
:1045680042c0b300824178000314a0000118a300e0
:104578000100320003417800824178000304a00062
:104588000128a30053053200834078008180fb0096
:10459800008070000070a0009440ab00feff3a005d
:1045a80000004000a041880000002c003428b7001b
:1045b800a04180008080d100808068004281de00b8
:1045c800810069004381de00810069004481de00ca
:1045d800810069004581de00810069004681de00b6
:1045e800810069004781de00810069004881de00a2
:1045f800810069004981de00810069004a81de008e
:10460800810069004b81de00810069004c81de0079
:1046180001016900cd81de004e80de00e10060000e
:104628000280690061006000808f500001003a003c
:1046380035a8a80000012000904188009801e200f8
:10464800bcfd32009801e200fcff3a00b9fd3700da
:10465800404b80000000e000fdff3200204b80004e
:104668006301400002014100439620006301790084
:104678000000e800f307280003006000440333004b
:10468800204b8800404b80000000e900404b880028
:1046980080822000024878002c28ef002ec8bf0036
:1046a8000080fb000041eb000008a300010032007d
:1046b80042c0b300824178000314a0000018a30090
:1046c8000100320003417800824178000304a00011
:1046d8000028a30001003200034178000281fb009a
:1046e800020078000050a0009440ab00feff3a00a2
:1046f80000004000a041880000002c003428b700ca
:10470800a04180008081d100808169004282de0062
:1047180083016a004382de0083016a004482de006e
:1047280083016a004582de0083016a004682de005a
:1047380083016a004782de0083016a004882de0046
:1047480083016a004982de0083016a004a82de0032
:1047580083016a004b82de0083016a004c82de001e
:1047680003026a00cd82de004e80de00e1016000b7
:1047780004806a0061006000808f510001003a00e7
:1047880035a8a80000012000904188009801e200a7
:10479800feff3a009440a80028c8bf000080fb0034
:1047a8008041eb000008a3000100320003c8b300f9
:1047b800034278000464a0000018a300010032003e
:1047c80084417800034278000454a0000028a30024
:1047d8000100320084417800034278000444a000bc
:1047e8000038a300010032008441780003427800b9
:1047f8000434a0000048a30001003200844178007e
:10480800034278000424a0000058a30001003200ed
:1048180084417800034278000414a0000068a300d3
:104828000100320084417800034278000404a000ab
:104838004700de0001003200844178000380fb005d
:104848004400dd00020070009440ab00feff3a0017
:1048580000004000a041880000002c003428b70068
:10486800a04180000081d10000016900c281de0002
:1048780002816900c381de0002816900c481de0013
:1048880002816900c581de0002816900c681de00ff
:1048980002816900c781de0002816900c881de00eb
:1048a80002816900c981de0002816900ca81de00d7
:1048b80002816900cb81de0002816900cc81de00c3
:1048c800828169004d82de004e80de006101600059
:1048d80003006a0061006000800f510001003a0087
:1048e80035a8a80000012000904188009801e20046
:1048f800feff3a009440a800830020000804e0006e
:1049080001003a008001eb000180fb000041eb0050
:104918000008a3000100320042c0b3000242780040
:104928000414a0000018a30001003200044178001c
:10493800024278000404a0000028a300010032000d
:10494800044178000280fb008301700000482000c9
:10495800030070009440ab00feff3a0000004000e6
:10496800a041880000002c003428b700a041800036
:104978000081d10000016900c281de000281690066
:10498800c381de0002816900c481de000281690002
:10499800c581de0002816900c681de0002816900ee
:1049a800c781de0002816900c881de0002816900da
:1049b800c981de0002816900ca81de0002816900c6
:1049c800cb81de0002816900cc81de008281690032
:1049d8004d82de004e80de006101600003006a0047
:1049e80061006000800f510001003a0035a8a8005e
:1049f80000012000904188009801e200feff3a0083
:104a08009440a80028c8bf000080fb00801f7800e1
:104a180010472900801f780081bf9f00cbf1070055
:104a280028c8bf00e4875700afb89700ee4f500082
:104a3800210432002868ef002ffd37008180fb0039
:104a48002ec8bf000000fb000000e800808f500067
:104a5800cd0332005cc8bf00e14f50006dfc3a0046
:104a6800800020000804e00001003a000000eb008c
:104a78000041eb000108a3000100320042c0b3006e
:104a8800824178000314a0000118a300010032003d
:104a980003417800824178000304a0000128a300a4
:104aa80001003200034178008280fb000080700022
:104ab80000a0a0009440ab00feff3a0000004000b8
:104ac800a041880000002c003428b700a0418000d5
:104ad8008080d100808068004281de00810069000a
:104ae8004381de00810069004481de0081006900a5
:104af8004581de00810069004681de008100690091
:104b08004781de00810069004881de00810069007c
:104b18004981de00810069004a81de008100690068
:104b28004b81de00810069004c81de0001016900d3
:104b3800cd81de004e80de00e10060000280690069
:104b480061006000808f500001003a0035a8a8007d
:104b580000012000904188009801e20075fc3200b5
:104b68009801e200fcff3a0072fc37008180fb00ec
:104b78002ec8bf000000fb000000e800808f500036
:104b88007a0332005cc8bf00e14f500021fc3a00b4
:104b9800830020000804e00001003a008001eb00d7
:104ba8000041eb000108a3000100320042c0b3003d
:104bb800024078000014a0000118a3000100320090
:104bc80000417800024078000004a0000128a300fa
:104bd80001003200004178000280fb0000b0a00014
:104be800008071009440ab00feff3a0000004000d6
:104bf800a041880000002c003428b700a0418000a4
:104c08008080d100808068004281de0081006900d8
:104c18004381de00810069004481de008100690073
:104c28004581de00810069004681de00810069005f
:104c38004781de00810069004881de00810069004b
:104c48004981de00810069004a81de008100690037
:104c58004b81de00810069004c81de0001016900a2
:104c6800cd81de004e80de00e10060000280690038
:104c780061006000808f500001003a0035a8a8004c
:104c880000012000904188009801e20029fc3200d0
:104c98009801e200fcff3a0026fc37005cc8bf0020
:104ca800e14f5000dbfb3a002ec8bf000080fb003c
:104cb8008040eb000008a3000100320041c0b300af
:104cc800014178000214a0000018a300010032007e
:104cd80082407800014178000204a0000028a30067
:104ce80001003200824078008180fb009440ab00d4
:104cf800feff3a0001804000a041880000002c001f
:104d08003428b700a04180000081d100000169006b
:104d1800c281de0002816900c381de000281690070
:104d2800c481de0002816900c581de00028169005c
:104d3800c681de0002816900c781de000281690048
:104d4800c881de0002816900c981de000281690034
:104d5800ca81de0002816900cb81de000281690020
:104d6800cc81de00828169004d82de004e80de004b
:104d78006101600003006a0061006000800f51005b
:104d880001003a0035a8a8000001200090418800e1
:104d98009801e200feff3a009440a800800020003d
:104da8000804e00001003a000000eb0002a0200027
:104db80081007100010070009440ab00feff3a00d2
:104dc80000004000a041880000002c003428b700f3
:104dd800a04180008080d100808068004281de0090
:104de800810069004381de00810069004481de00a2
:104df800810069004581de00810069004681de008e
:104e0800810069004781de00810069004881de0079
:104e1800810069004981de00810069004a81de0065
:104e2800810069004b81de00810069004c81de0051
:104e380001016900cd81de004e80de00e1006000e6
:104e48000280690061006000808f500001003a0014
:104e580035a8a80000012000904188009801e200d0
:104e6800b4fb32009801e200fcff3a00b1fb3700c6
:104e7800e14f5000d3fb3a009440ab00feff3a00ec
:104e8800402c2000a041880000002c003428b700e6
:104e9800a04180008080d100808068004281de00cf
:104ea800810069004381de00810069004481de00e1
:104eb800810069004581de00810069004681de00cd
:104ec800810069004781de00810069004881de00b9
:104ed800810069004981de00810069004a81de00a5
:104ee800810069004b81de00810069004c81de0091
:104ef80001016900cd81de004e80de00e100600026
:104f08000280690061006000808f500001003a0053
:104f180035a8a80000012000904188009801e2000f
:104f2800feff3a009440a8009440ab00feff3a0010
:104f380040902000a041880000002c003428b700d1
:104f4800a04180008080d100808068004281de001e
:104f5800810069004381de00810069004481de0030
:104f6800810069004581de00810069004681de001c
:104f7800810069004781de00810069004881de0008
:104f8800810069004981de00810069004a81de00f4
:104f9800810069004b81de00810069004c81de00e0
:104fa80001016900cd81de004e80de00e100600075
:104fb8000280690061006000808f500001003a00a3
:104fc80035a8a80000012000904188009801e2005f
:104fd800feff3a009440a8009440ab00feff3a0060
:104fe80040862000a041880000002c003428b7002b
:104ff800a04180008080d100808068004281de006e
:10500800810069004381de00810069004481de007f
:10501800810069004581de00810069004681de006b
:10502800810069004781de00810069004881de0057
:10503800810069004981de00810069004a81de0043
:10504800810069004b81de00810069004c81de002f
:1050580001016900cd81de004e80de00e1006000c4
:105068000280690061006000808f500001003a00f2
:1050780035a8a80000012000904188009801e200ae
:10508800feff3a009440a8009440ab00feff3a00af
:1050980040f02000a041880000002c003428b70010
:1050a800a04180008080d100808068004281de00bd
:1050b800810069004381de00810069004481de00cf
:1050c800810069004581de00810069004681de00bb
:1050d800810069004781de00810069004881de00a7
:1050e800810069004981de00810069004a81de0093
:1050f800810069004b81de00810069004c81de007f
:1051080001016900cd81de004e80de00e100600013
:105118000280690061006000808f500001003a0041
:1051280035a8a80000012000904188009801e200fd
:10513800feff3a009440a8009440ab00feff3a00fe
:1051480040e02100a041880000002c003428b7006e
:10515800a04180008080d100808068004281de000c
:10516800810069004381de00810069004481de001e
:10517800810069004581de00810069004681de000a
:10518800810069004781de00810069004881de00f6
:10519800810069004981de00810069004a81de00e2
:1051a800810069004b81de00810069004c81de00ce
:1051b80001016900cd81de004e80de00e100600063
:1051c8000280690061006000808f500001003a0091
:1051d80035a8a80000012000904188009801e2004d
:1051e800feff3a009440a80080062000801f780047
:1051f800d0452900801f7800d4ef07005cc8bf00a5
:10520800e48757000004e00082fa3200effa370022
:1052180002c0e800840020000804e00001003a0011
:105228000002eb008180fb008041eb000108a30035
:105238000100320043c0b300034178000214a0000b
:105248000118a30001003200824178000341780070
:105258000204a0000128a300010032008241780066
:105268000080fb008040eb000008a3000100320032
:1052780001c8b300014178000264a0000018a3002f
:105288000100320082407800014178000254a000f9
:105298000028a30001003200824078000141780014
:1052a8000244a0000038a3000100320082407800c8
:1052b800014178000234a0000048a3000100320038
:1052c800824078008180fb00c408dd000380fb0079
:1052d80001007000000072009440ab00feff3a002d
:1052e80000004000a041880000002c003428b700ce
:1052f800a04180008080d100808068004281de006b
:10530800810069004381de00810069004481de007c
:10531800810069004581de00810069004681de0068
:10532800810069004781de00810069004881de0054
:10533800810069004981de00810069004a81de0040
:10534800810069004b81de00810069004c81de002c
:1053580001016900cd81de004e80de00e1006000c1
:105368000280690061006000808f500001003a00ef
:1053780035a8a80000012000904188009801e200ab
:105388006cfa32009801e200fcff3a0069fa370033
:105398000000e90003f82f00008071000000e80019
:1053a800b7fc37002e48ec00004178000281fb0072
:1053b8000040eb000208a3000100320040c0b30027
:1053c800804178000314a0000218a30001003200f5
:1053d80003407800804178000304a0000228a3005d
:1053e80001003200034078000080fb000040a0006c
:1053f8009440ab00feff3a0000004000a041880046
:1054080000002c003428b700a04180000081d100a2
:1054180000016900c281de0002816900c381de00eb
:1054280002816900c481de0002816900c581de0055
:1054380002816900c681de0002816900c781de0041
:1054480002816900c881de0002816900c981de002d
:1054580002816900ca81de0002816900cb81de0019
:1054680002816900cc81de00828169004d82de0004
:105478004e80de006101600003006a006100600088
:10548800800f510001003a0035a8a8000001200053
:10549800904188009801e200feff3a009440a8007d
:1054a8008904e800b0482900801f780091bf9f0058
:1054b80026ef07008f87e900afb897003c08ab00dc
:1054c800a4fb3a00f44180000408a300a1fb3200c9
:1054d8002e48ec00004178000281fb000040eb0000
:1054e8000208a3000100320040c0b30080417800e8
:1054f8000314a0000218a300010032000340780042
:10550800804178000304a0000228a30001003200b3
:10551800034078000080fb00028120000000710039
:105528009440ab00feff3a0000004000a041880014
:1055380000002c003428b700a04180000081d10071
:1055480000016900c281de0002816900c381de00ba
:1055580002816900c481de0002816900c581de0024
:1055680002816900c681de0002816900c781de0010
:1055780002816900c881de0002816900c981de00fc
:1055880002816900ca81de0002816900cb81de00e8
:1055980002816900cc81de00828169004d82de00d3
:1055a8004e80de006101600003006a006100600057
:1055b800800f510001003a0035a8a8000001200022
:1055c800904188009801e200feff3a009440a8004c
:1055d8008904e80040492900801f780091bf9f0096
:1055e800daee07008f87e900afb8970059fb37005c
:1055f80000412000060370009440ab00feff3a0013
:1056080006034300a641880000002c003428b70098
:10561800a04180000081d10000016900c281de0044
:1056280002816900c381de0002816900c481de0055
:1056380002816900c581de0002816900c681de0041
:1056480002816900c781de0002816900c881de002d
:1056580002816900c981de0002816900ca81de0019
:1056680002816900cb81de0002816900cc81de0005
:10567800828169004d82de004e80de00610160009b
:1056880003006a0061006000800f510001003a00c9
:1056980035a8a80000012000904188009801e20088
:1056a800feff3a009440a80090472900801f780028
:1056b80091bf9f00a5ee0700e54180000501780035
:1056c8008f87e900afb897000518a300f3003200f0
:1056d800f4418000490020001afb37005cc8bf0075
:1056e800e14f5000b5f93a000281fb000040eb00a1
:1056f8000208a3000100320040c0b30080417800d6
:105708000314a0000218a30001003200034078002f
:10571800804178000304a0000228a300f7003200ab
:10572800034178000281fb0000ccb3005a48b40062
:105738000080fb008041eb000008a300010032005c
:1057480003c8b300034278000464a0000018a30053
:105758000100320084417800034278000454a0001c
:105768000028a30001003200844178000342780039
:105778000444a0000038a3000100320084417800ee
:10578800034278000434a0000048a300010032005e
:1057980084417800034278000424a0000058a30044
:1057a8000100320084417800034278000414a0000c
:1057b8000068a300010032008441780003427800a9
:1057c8000404a0004700de00c7003200044078004f
:1057d8000080fb004400dd00000071009440ab0035
:1057e800feff3a0000004000a041880000002c00a5
:1057f8003428b700a04180008081d10080816900f1
:105808004282de0083016a004382de0083016a006f
:105818004482de0083016a004582de0083016a005b
:105828004682de0083016a004782de0083016a0047
:105838004882de0083016a004982de0083016a0033
:105848004a82de0083016a004b82de0083016a001f
:105858004c82de0003026a00cd82de004e80de004c
:10586800e101600004806a0061006000808f5100df
:1058780001003a0035a8a8000001200090418800e6
:105888009801e200feff3a009440a8009440ab0063
:10589800feff3a0002014100a241880000002c00ee
:1058a8003428b700a04180000081d10000016900c0
:1058b800c281de0002816900c381de0002816900c5
:1058c800c481de0002816900c581de0002816900b1
:1058d800c681de0002816900c781de00028169009d
:1058e800c881de0002816900c981de000281690089
:1058f800ca81de0002816900cb81de000281690075
:10590800cc81de00828169004d82de004e80de009f
:105918006101600003006a0061006000800f5100af
:1059280001003a0035a8a800000120009041880035
:105938009801e200feff3a009440a800f00d200014
:10594800801f7800d0452900801f780081bf9f0004
:10595800feed07005cc8bf00e4875700afb89700aa
:10596800e2cf500017f93a0041fd37005c68ef00bc
:105978004f0678004f05be004f04be000080fa00b5
:1059880000000600a8f8370010c0b3005ce8b700b4
:1059980033fc37002e48ec000080fb00e104600077
:1059a8000043eb000100320046c0b3000645780012
:1059b8000a14a0008083d1000708a30001003a0060
:1059c800064578008a4578000b04a0004283de0073
:1059d8000608a3003b0032000b4078000080fb0063
:1059e80000a0a0009440ab00feff3a000000400079
:1059f800a041880000002c003428b700a041800096
:105a08000085d10000056d00c285de000a856d00a5
:105a1800c385de000a856d00c485de000a856d0039
:105a2800c585de000a856d00c685de000a856d0025
:105a3800c785de000a856d00c885de000a856d0011
:105a4800c985de000a856d00ca85de000a856d00fd
:105a5800cb85de000a856d00cc85de008a856d0069
:105a68004d86de004e80de00610560000b006e0092
:105a780061006000800f550001003a0035a8a800b9
:105a880000012000904188009801e20068f9320086
:105a98009801e200fcff3a0065f937004900200050
:105aa800f3418000030278000418a30015003a00af
:105ab8008202780023fa3700f0c0b30028e8b70064
:105ac8000df937000a4078000080fb0000a0a00014
:105ad800c4ff3700824078008180fb00008070009e
:105ae8000070a000acfa3700034078000080fb008b
:105af8004400dd000000710038ff370000417800e5
:105b080008ff37002e48ec00004178000281fb00b6
:105b18000040eb000208a3000100320040c0b300bf
:105b2800804178000314a0000218a300010032008d
:105b380003407800804178000304a0000228a300f5
:105b480001003200034078000080fb0002c1200001
:105b5800000071009440ab00feff3a0000004000d6
:105b6800a041880000002c003428b700a041800024
:105b78000081d10000016900c281de000281690054
:105b8800c381de0002816900c481de0002816900f0
:105b9800c581de0002816900c681de0002816900dc
:105ba800c781de0002816900c881de0002816900c8
:105bb800c981de0002816900ca81de0002816900b4
:105bc800cb81de0002816900cc81de008281690020
:105bd8004d82de004e80de006101600003006a0035
:105be80061006000800f510001003a0035a8a8004c
:105bf80000012000904188009801e200feff3a0071
:105c08009440a8008904e80020482900801f7800f3
:105c180091bf9f004ded0700e5418000f4418000f1
:105c28008f87e900afb89700c6f9370010438000a6
:105c380000000600104380000000e000fdff320075
:105c4800f14280006380400000004000e2852000af
:105c5800620078008100e800f20728008280600076
:105c68000d003300f14288000600fc00120280009b
:105c7800020eb30012028800114380008100e9007f
:105c8800114388000600fc0011028000f141b200b7
:105c980011028800000006008100e90002f82f00c8
:105ca800810071008100e800f14288000600fc00d4
:105cb80012028000020eb300120288001143800015
:105cc8008100e900114388000600fc0011028000f1
:105cd800f141b2001102880000000600eeff370013
:105ce8008080fb000040eb000108a30001003200a7
:105cf80000c8b300004178000264a0000118a300a6
:105d08000100320002407800004178000254a000ef
:105d18000128a30001003200024078000041780009
:105d28000244a0000138a3000100320002407800bc
:105d3800004178000234a0000148a30001003200ad
:105d480002407800004178000224a0000158a30016
:105d58000100320002407800004178000214a000df
:105d68000168a30001003200024078000041780079
:105d78000204a000c708de000100320002407800db
:105d8800000006008080fb000040eb000108a30033
:105d98000100320040c0b300004178000214a000a6
:105da8000118a30001003200024078000041780089
:105db8000204a0000128a30001003200024078007c
:105dc80000000600840020000004e00001003a0002
:105dd8000002eb008180fb008041eb000108a3007a
:105de8000100320043c0b300034078000014a00053
:105df8000118a300010032008041780003407800b8
:105e08000004a0000128a3000100320080417800ae
:105e18000280fb008040eb000008a3000100320074
:105e280001c8b300014178000264a0000018a30073
:105e38000100320082407800014178000254a0003d
:105e48000028a30001003200824078000141780058
:105e58000244a0000038a30001003200824078000c
:105e6800014178000234a0000048a300010032007c
:105e780082407800014178000224a0000058a30065
:105e88000100320082407800014178000214a0002d
:105e98000068a300010032008240780001417800c8
:105ea8000204a0004700de000100320082407800b2
:105eb8000180fb004400dd008381fb00008071004d
:105ec800000072009440ab00feff3a000000400062
:105ed800a041880000002c003428b700a0418000b1
:105ee8008080d100808068004281de0081006900e6
:105ef8004381de00810069004481de008100690081
:105f08004581de00810069004681de00810069006c
:105f18004781de00810069004881de008100690058
:105f28004981de00810069004a81de008100690044
:105f38004b81de00810069004c81de008100690030
:105f48004d81de004e80de00610060008100690046
:105f5800e1806000810f500001003a0035a8a800d8
:105f680000012000904188009801e200feff3a00fd
:105f78009440a800100005009440ab00feff3a00d2
:105f880000004000a041880000002c003428b70021
:105f9800a04180008080d100808068004281de00be
:105fa800810069004381de00810069004481de00d0
:105fb800810069004581de00810069004681de00bc
:105fc800810069004781de00810069004881de00a8
:105fd800810069004981de00810069004a81de0094
:105fe800810069004b81de00810069004c81de0080
:105ff800810069004d81de004e80de006100600096
:1060080081006900e1806000810f500001003a00c2
:1060180035a8a8000001200090418800c00c80002d
:106028000000e000fdff3a009440a80000000600d0
:1060380000417800404b8000f1072000810f50009c
:106048000d003c000000e800404b8800314b800008
:106058008201fb006381400002014100409620005c
:10606800033079000100e800f10728008100600092
:1060780002003300314b8800000006008100e9006f
:1060880002f82f00810071008100e800314b880080
:10609800f9ff3700404b800000000600404b8000ad
:1060a8000000e000fdff3200214b800063804000cb
:1060b8000000400042962000620078008100e8005d
:1060c800f20728008280600005003300214b880019
:1060d800414b80008100e900414b88000000060028
:1060e8008100e90002f82f00810071008100e800ba
:1060f800214b8800414b80008100e900414b88001a
:1061080000000600f6ff3700889fbe008a9fbe0089
:106118008c9fbe002f0607000000e00005003a0033
:106128000000eb004f06be004f05be004f04be0046
:106138000000060029060700f34f5000480032000f
:10614800f44f500021003200b14280000100e0000d
:10615800110032008100e800b14288000108a30064
:1061680047003200a142800062fa2000e2c17800b4
:106178000340700000f178008100e800a142880027
:106188000000eb004f06be004f05be004f04be00e6
:1061980000000600e7ff3700a142800062fa2000f5
:1061a80000f178008100e800a1428800100020007a
:1061b800b04288000000eb004f06be004f05be004d
:1061c8004f04be0000000600daff37005428ef0035
:1061d8005628ef006cfa20001c407800e84f500069
:1061e80032003200e44f5000cdff3a0070fa200030
:1061f8001040780081fa20009140780092fa20003f
:10620800124178000104e00056003a000204e00060
:1062180054003a000000fb001208e30009003200b5
:106228000008a300c10032003c08a8000018a30021
:10623800b90032003c28a80011c0b300a382200096
:1062480081497800904088000000eb004f06be00ae
:106258004f05be004f04be0000000600b5ff370022
:106268005428ef005628ef000000eb004f06be0050
:106278004f05be004f04be0000000600adff37000a
:106288000000fb004400dd0062fa2000a14280000b
:1062980000f178000000eb004f06be004f05be007d
:1062a8004f04be0000000600a2ff37000c00e80003
:1062b8009046780063004600904478000904e000a6
:1062c8009c003400704080000000e0002e00320086
:1062d8000000e000020034000904e0007f00320002
:1062e8000d04fb0080408000800f5400190032002c
:1062f800881f7800801f780050ae2900801f780022
:1063080092eb07008240800008006900e68757008a
:106318000008a3005e003a000018a30049003a00f4
:106328000028a30036003a000048a3000800320005
:106338000848a3008100320010002000a040880017
:1063480000b52900801f780080eb07008f87e900df
:10635800884088001c407800e44f500070ff3a00e5
:10636800a2ff37008100fb00e14088008200fb00ab
:106378008100ea00f140880011c0b300a382200028
:1063880081497800a3ff37008904fb00891f780042
:10639800e0ac2900801f78006ceb0700794088008a
:1063a80088b62900ca12200008054500e48757006e
:1063b8001880fb00808f54000600320063044400fc
:1063c8008a0f5400c6ff32001880fb00808f5400eb
:1063d800faff3a001408e20049003200a84590008c
:1063e8000b40780012ff0700008220000b4878005d
:1063f800630444008a0f5400f3ff3a00b8ff3700e3
:10640800e4046400891f780080b32900801f7800a5
:106418004eeb0700e48757000900e00059003200fe
:1064280000b12900801f780048eb070060c0b30066
:10643800fffe070081408000088068008f87e90020
:10644800b9ff3700e2046400891f7800e0b1290031
:10645800801f78003deb0700e48757000900e00043
:106468005100320000b12900801f780037eb070087
:10647800a0c0b300eefe070082408000080069005b
:106488008f87e9000028a300a7ff3200dcff370050
:10649800e1046400891f780070af2900801f78002c
:1064a8002aeb0700e48757000900e0002a003200c1
:1064b80000b12900801f780024eb0700c0c0b3009a
:1064c800dbfe070083408000088069008f87e900b1
:1064d8000018a30092ff3200daff3700801f78000f
:1064e80090ad2900801f780018eb07000e28ef00f8
:1064f8002048ec00cefe0700e487570078ff3700fd
:10650800984590000b407800c9fe070000822000e3
:106518000b487800b6ff37003c28a90011c0b3002b
:10652800a38220008149780046ff37003c08a90073
:106538003eff37007040800065ff37001428ef00e9
:10654800b0b52900801f780000eb07008f87e900ad
:10655800884088007fff370060b12900801f7800dd
:10656800faea0700d0c0b300b1fe070081408000fe
:10657800088068008f87e9000018a30068ff3200d0
:10658800b0ff370060b12900801f7800efea0700ec
:1065980070c0b300a6fe07008240800008006900b2
:1065a8008f87e90060ff370060b12900801f7800fd
:1065b800e6ea0700b0c0b3009dfe070083408000f4
:1065c800088069008f87e9000028a30056ff320081
:1065d8008bff3700889fbe008a9fbe008c1f780003
:1065e80010469000b04490000904e0004d003400cb
:1065f800704080000000e000260032000000e0004b
:10660800020034000904e000800032000c04fb00a2
:1066180080408000800f540019003200881f7800e5
:10662800801f780050ae2900801f7800c7ea070055
:106638008140800008806800e68757000008a300b2
:106648004d003a000018a3005d003a000028a3009e
:1066580036003a000048a300080032000848a300aa
:106668007300320010002000a040880000b5290007
:10667800801f7800b5ea07008f87e9008840880006
:10668800100020004f0678004f05be004f04be00e2
:10669800000006008904fb00891f7800e0ac29008f
:1066a800801f7800a9ea07007940880088b6290089
:1066b800ca12200008054500e48757001880fb002f
:1066c800808f540006003200630444008a0f54008f
:1066d800ceff32001880fb00808f5400faff3a008a
:1066e8001408e20009003200a84590000b40780029
:1066f8004ffe0700008220000b4878006304440026
:106708008a0f5400f3ff3a00c0ff37009845900005
:106718000b40780046fe0700008220000b487800f6
:10672800f6ff370070408000b4ff3700e4046400cf
:10673800891f780080b32900801f780083ea07004a
:10674800e48757000900e0004b00320000b129003f
:10675800801f78007dea070060c0b30034fe0700a0
:1067680081408000088068008f87e9000048a30006
:10677800c2ff3200b9ff3700e1046400891f7800c6
:1067880070af2900801f780070ea0700e48757007f
:106798000900e0004300320000b12900801f7800a2
:1067a8006aea0700c0c0b30021fe070081408000ec
:1067b800088068008f87e9000018a300a3ff320053
:1067c800e2046400891f7800e0b12900801f780086
:1067d8005eea0700e48757000900e0001b0032006a
:1067e80000b12900801f780058ea0700a0c0b30054
:1067f8000ffe070081408000088068008f87e9004d
:106808000028a30093ff3200c8ff3700801f7800dc
:1068180090ad2900801f78004cea07000e28ef0091
:106828002048ec0002fe0700e487570077ff370096
:106838001428ef00b0b52900801f780043ea07004c
:106848008f87e900884088008dff370060b12900f4
:10685800801f78003dea0700b0c0b300f4fd0700d0
:1068680081408000088068008f87e9000028a30025
:1068780078ff3200adff370060b12900801f780033
:1068880032ea070070c0b300e9fd070081408000cc
:10689800088068008f87e9000048a30077ff32006e
:1068a8006eff370060b12900801f780027ea0700d3
:1068b800d0c0b300defd070081408000088068007a
:1068c8008f87e9000018a30060ff3200bcff370083
:1068d80090419000a0409000304190000104e000f9
:1068e80010003a000204e0000e003a000300fb002a
:1068f8001208e300090032000008a300110032006a
:106908003c08a8000018a300110032003c28a80089
:1069180011c0b300a282200001497800904088008d
:10692800100005008100fb00e14088000201fb0027
:106938000201ea00f240880010c0b3002ae8b7005c
:10694800eaff37003c08a9000018a300efff3a004f
:106958003c28a90011c0b300a28220000149780098
:10696800eeff3700a06b800000000600a06b8000df
:106978000000e000fdff3200816b80006380400072
:106988000000400002d72000620078008100e80083
:10699800f2072800828060000e003300816b8800b7
:1069a8000600fc0012028000020eb30012028800ea
:1069b800a16b80008100e900a16b88000600fc0043
:1069c80011028000f141b20011028800f00fb200fc
:1069d800000006008100e90002f82f008100710024
:1069e8008100e800816b88000600fc00120280002c
:1069f800020eb30012028800a16b80008100e9003a
:106a0800a16b88000600fc0011028000f141b20071
:106a180011028800f00fb20000000600edff3700f9
:106a28000000fb0080004000414288004928a9007e
:106a38000081d10000016900c280de000281680087
:106a4800c380de0002816800c480de000281680025
:106a5800c580de0002816800c680de000281680011
:106a680061016100cf00de004f00de000000690018
:106a7800808f5000010032004928a800b000200093
:106a88003042880097a0a9001000200050428800da
:106a9800d122a900d102a900d502a90000f0200046
:106aa8000100200044040700d522a900001420009a
:106ab800010020004004070097a0a800d102a80008
:106ac80000000600889fbe008a9fbe008c9fbe0003
:106ad8002ca3ef00d122a800d102a800d062a900ff
:106ae800d702a800d722a80000fe2f008206b60011
:106af8008001b3001034880087a0a900f0f82f00a7
:106b0800b200b6000006b300900588008240a900d4
:106b1800b0002000104288004428ef00304288006e
:106b28004828ef004a28ef004028ef00d462a80068
:106b380000402d00010320001f04070087a0a900c2
:106b480097a0a80040c92900801f7800d0c9290053
:106b5800801f780090ca2900801f78007be9070011
:106b6800e687570029002000480620000cd720009f
:106b7800fb072800eacc29000df82f00a06b800045
:106b88000000e00010003a0000202e004100200024
:106b9800090407000804e9000900e0002d0032009c
:106ba8000800e000f5ff3a0060cd2900801f78005a
:106bb80066e907008f87e9004f06be004f05be0053
:106bc8004f04be0000000600a06b80000000e0003b
:106bd800fdff3200816b80006380400000004000b0
:106be8006c0178000100e8000b0060007f003300b2
:106bf800806b88000400fc00000e20004220b700d3
:106c0800a06b80000000e900a06b88000600fc0073
:106c180010028000f041b2001002880002007800e3
:106c2800f00fb200801f7800891f78008a1f780053
:106c380046e907008904e900e687570000202e008e
:106c480041002000dc0307000804e9000900e00017
:106c5800d3ff3a000800e000d3ff3200e0ff2f0026
:106c6800404288004928a9004928a800b00020000f
:106c78003042880097a0a9001000200050428800e8
:106c8800d122a900d102a900d502a90000f0200054
:106c980001002000c8030700d522a9000014200025
:106ca80001002000c403070097a0a800d102a80093
:106cb800883e2000390020000cd72000fb07280060
:106cc8009ace29000df82f00a06b80000000e0008c
:106cd8005d003a0000202e0041002000b6030700a6
:106ce8000900e000020032000804e900f6ff3a005b
:106cf80080fe2f00404288004928a900b0002000eb
:106d08003042880097a0a900100020005042880057
:106d1800d122a900d102a900d502a90000f02000c3
:106d280001002000a4030700d522a90000142000b8
:106d380001002000a003070097a0a800d102a80026
:106d4800a06b80000000e00009003a00883e2000a7
:106d580000202e004100200097030700a06b800050
:106d68000000e00002003a000804e900f8ff3a00d9
:106d7800a06b80000000e0008fff3200a06b800055
:106d88000000e000fdff3200806b8000e30040005f
:106d98008180400002d72000e28078000000e800ef
:106da800f1072800010060005a003300806b88005a
:106db8000400fc00000e20004220b700a06b8000f9
:106dc8000000e900a06b88000600fc0010028000ab
:106dd800f041b200100288004f06be004f05be0009
:106de8004f04be000000060077ff37000000e900ee
:106df800008076000000e800806b88000400fc003a
:106e0800000e20004220b700a06b80000000e900bf
:106e1800a06b88000600fc0010028000f041b20060
:106e28001002880002007800f00fb200801f78007e
:106e3800891f78008a1f7800c4e807008904e900e0
:106e4800e68757007dff3700a06b80000000e00058
:106e5800fdff3200816b800063804000000040002d
:106e68006c0178000100e8000b006000130033009b
:106e7800806b88000400fc00000e20004220b70050
:106e8800a06b80000000e900a06b88000600fc00f1
:106e980010028000f041b200100288000200780061
:106ea800f00fb200801f78008a1f7800a7e807005b
:106eb8008904e900e487570086ff37000000e900ed
:106ec800008076000000e800806b88000400fc0069
:106ed800000e20004220b700a06b80000000e900ef
:106ee800a06b88000600fc0010028000f041b20090
:106ef8001002880002007800f00fb200801f7800ae
:106f08008a1f780091e807008904e900e4875700a0
:106f180070ff37000000e90001f82f0000807000c2
:106f28000000e800806b88000400fc00000e2000d0
:106f38004220b700a06b80000000e900a06b880029
:106f48000600fc0010028000f041b2001002880028
:106f5800a1ff3700b0002000104288004428ef004d
:106f6800304288004828ef004a28ef004028ef0008
:106f7800000006002dfb0700800078000000eb00f1
:106f88000100e00001003a000000060029fb0700ac
:106f980000408800f1ff20000101600012408800d5
:106fa800670060003040880076fb07000080fb0027
:106fb8003040880010408000e8006000c388de0090
:106fc800414088004400de00f00fb20050408800c5
:106fd80043fb0700004178000280fb002040880046
:106fe8004140800001f0a7008100ea000100ea00aa
:106ff8004f00de006180200091407800f3f2070026
:1070080010000500889fbe008a9fbe009d020700f1
:10701800800078000000eb000100e00003003a0067
:107028004f05be004f04be0000000600970207008f
:1070380010418800cde2a900cdc2a9000e28ef00ba
:10704800110e2000810f50005b003200010e20005d
:10705800810f500046003200010f2000810f5000c0
:1070680036003200714080000100e000020032006a
:107078000100400010418800cdc2ab00130032006f
:1070880010002000b0408800d8922900491a20003a
:10709800888444000b0028004a8e2900e30054002d
:1070a80010418000910f10000f003200640444006a
:1070b800890f5400f9ff3a00100020004f05be0068
:1070c8004f04be0000000600d8ff37001628ef0066
:1070d800d8922900491a2000888444000b0028000f
:1070e8004a8e2900edff37001408e20047003200fd
:1070f8001800fb002041880062168000828065002d
:10710800020032000000e80020418800c8fb0700a8
:1071180020418000f00fb200801f78002208f8009c
:107128008a1f780009e80700e687570064044400ce
:10713800890f5400d9ff3a00dfff3700cde2a800dd
:107148005202070010418800cdc2ab00c5ff3200d3
:107158001608e20031003a002228ef000000eb0098
:10716800714080000100e000c3ff3200c0ff37001b
:10717800cdc2a80000002e0070408800430207001e
:1071880010418800f40f5000b3ff3a0010002000af
:10719800a0408800f08c2900801f7800ebe70700ea
:1071a800104180008f87e900010f2000810f5000f7
:1071b800acff3a00e1ff3700008c2900801f7800ff
:1071c800e2e707000e28ef0040112e00104188006a
:1071d800c0c9b30028e8b7002c0207002b0207003b
:1071e8002a020700290207002802070027020700d1
:1071f80026020700104180008f87e900010e200059
:10720800810f500094ff3a00d9ff370078f89700b3
:107218000000fb0020418800b7ff3700f40f500042
:1072280090ff3a001428ef00908d2900801f780005
:10723800c6e707008f87e900100020004f05be0051
:107248004f04be000000060078ff3700889fbe008c
:107258008a1f7800c3fd0700800078000000eb005b
:107268000100e00003003a004f0578004f04be001b
:1072780000000600bdfd070026e8b700c1408000f9
:10728800e8fd200000f478008100e800c140880093
:1072980010002000e28f5000f3ff34008884e800db
:1072a8001980fb00801f78000805e8001a80fb00a1
:1072b800801f78001880fb00801f7800508f2900fd
:1072c800801f7800a1e707001a00fb00e040880053
:1072d8009900fb00f140880098417800c2832000a3
:1072e80003497800e88757003c68ab000f0032007c
:1072f800811f7800801f7800e0912900801f7800a6
:1073080092e707001828ef00e687570010002000d2
:107318003c68ab00d4ff32002ae8b7004f0578007c
:107328004f04be0000000600d2ff3700a0902900dd
:10733800801f780085e707004008ec0000428800bd
:107348008f87e9000000e0000200340001ff070019
:107358004028ef00f1408000e0408000e4ff370063
:10736800889fbe00f0f32f004427b600f08f2f004f
:107378004427b600d062a90065010700b0f10700f4
:10738800ef010700cffd0700f9ff200008ff2000ec
:1073980026fa07000000e0000c003a008d01070003
:1073a8000000e0000400320057fb070089010700d5
:1073b8000000e000fcff3a0012ff0700a3ff0700ef
:1073c8001afa07000000e000f4ff320019fa07007b
:1073d8000040880089006000114088006700600054
:1073e8003040880067fa07000080fb0030408800c2
:1073f80010408000e8006000c388de00414088003b
:10740800080060004480de005040880034fa07001d
:10741800004178000280fb00204088004140800045
:1074280001f0a7008100ea000100ea004f00de0039
:107438006180200091407800e4f10700d7ff370011
:08744800c4fe0700db01370060
:020000040000fa
:107450006a0a00000002000002000000a994ad00ca
:1074600094b19400b594b90094bd9400c194c50042
:1074700094c99400ce94d30094d89400dd94e20093
:1074800094e79400ec94f10094f69400fb940000cf
:10749000950595000a950a00950f95001495190019
:1074a000951e950023952800952d9500329537005f
:1074b000953c950041954600954b9500509555009b
:1074c000955a95005f956400956995006e957300d7
:1074d000957895007d958200958795008c95900014
:1074e0009594950098959c0095a09500a495a8006a
:1074f00095ac9500b095b40095b89500bc95c000ca
:1075000095c49500c895cc0095d09500d495d80029
:1075100095dc9500e095e40095e89500ec95f00089
:1075200095f49500f895fc009500960000960400ef
:10753000960896000c9610009614960018961c005b
:107540009620960024962800962c960030963400bb
:10755000963896003c9640009644960048964c001b
:107560009650960054965800965c9600609664007b
:10757000966896006c9670009674960078967c00db
:107580009680960084968800968c9600909694003b
:10759000969896009c96a00096a49600a896ac009b
:1075a00096b09600b496b80096bc9600c096c400fb
:1075b00096c89600cc96d00096d49600d896dc005b
:1075c00096e096002496e40096e89600ec96f0008b
:1075d00096f49600f896fc00960097000497080031
:1075e000970c970010971400971897001c9720008d
:1075f0009724970028972c009730970034973800ed
:10760000973c970040974400974897004c9750004c
:107610009754970058975c009760970064976800ac
:10762000976c970070977400977897007c9780000c
:107630009784970088978c0097909700949798006c
:10764000979c9700a097a40097a89700ac97b000cc
:1076500097b497007897b80097bc9700c097c4007c
:1076600097c89700cc97d00097d49700d897dc00a4
:1076700097e09700e497e80097ec9700f097f40004
:1076800097f89700fc9700009804980008980c0061
:107690009810980014981800981c980020982400be
:1076a000982898002c9830009834980038983c001e
:1076b0009840980044984800984c9800509854007e
:1076c000985898005c9860009864980068986c00de
:1076d0009870980074987800987c9800809884003e
:1076e000988898008c9890009894980098989c009e
:1076f00098a09800a498a80098ac9800b098b400fe
:1077000098b89800bc9800005e0800000c020000c9
:107710000000000028080000140000000000000025
:107720005a08000004000000020000001f000100d1
:1077300000000000de0f0000040000000000000058
:107740000008000028000000000000006a0c000093
:1077500006010000000000004c08000008000000c6
:1077600000000000700d0000060100000000000095
:107770003c0800001000000000000000fe0e0000a9
:107780008600000000000000a60f00001e000000a0
:107790000000000054080000060000000000000087
:1077a000760e0000880000000200000001000000ca
:1077b000009c0e009d0e9c000e9c0e009c0e9c00da
:1077c0000e8c0e0000000000000000000000000011
:1077d00000000000000000000000000000000000a9
:1077e000000208000101c4000ec50e00c40ec40052
:1077f0000ec40e00c40eb4000e0000000000000015
:107800000000000000000000000000000000000078
:10781000000000000000020008020200ec0eed0073
:107820000eec0e00ec0eec000eec0e00dc0e000078
:107830000000000000000000000000000000000048
:10784000000000000000000000000000760e9e0016
:107850000ec60e0000000000000000000000000046
:1078600000000000e60f0000020000000000000021
:10787000c40f00001a00000002000000686a6c00db
:10788000747a4c00000001000002000004000800af
:1078900000100000000020002b2d2300300000000d
:1078a000e80f0000020000000200000004000000d9
:1078b000e20f00000400000000000000840f000040
:1078c0002200000002000000303132003334350065
:1078d0003637380039414200434445004600300005
:1078e0003132330034353600373839006162630095
:1078f0006465660000000000ea0f0000020000005e
:107900000200000001000000ec0f00000200000077
:0879100000000000000000006f
:020000040000fa
:10791800c902a800c922a900d082a800c102a800f3
:1079280000fe2f00a806b6000030a00040358800f1
:10793800f10f2e004035800080806000004021005b
:107948000100700040358800007020004036880033
:107958000000eb0010788800f07788000078880035
:1079680045e2a90045c2a8004362a9004342a90014
:107978004322a8004302a90042e2a90042c2a9008a
:1079880042a2a900c00120004222b700c0ff2f0078
:107998004202b6000010a000101288004402a9009c
:1079a80040c2a9008540a9009540a800f08f2f008b
:1079b800a800b6000080a0004005880030fe2f0017
:1079c8004002b6000030a0000012880041e2a80082
:1079d8000000060010788000000006001078800083
:1079e8000000e000fdff3200f17780006680400073
:1079f800e2ef2000624078008100e800f2072800ea
:107a0800828060000d003300f17788000600fc00da
:107a180012028000020eb300120288001178800062
:107a28008100e900117888000600fc00110280003e
:107a3800f141b20011028800000006008100e9004f
:107a480002f82f00810071008100e800f1778800ba
:107a58000600fc0012028000020eb3001202880029
:107a6800117880008100e900117888000600fc0088
:107a780011028000f141b2001102880000000600e6
:107a8800eeff37007063800000000600706380001e
:107a98000000e000fdff3200516380006380400079
:107aa80000004000a2c62000620078008100e800c3
:107ab800f2072800828060000e00330051638800be
:107ac8000600fc0012028000020eb30012028800b9
:107ad800716380008100e900716388000600fc0082
:107ae80011028000f141b20011028800f00fb200cb
:107af800000006008100e90002f82f0081007100f3
:107b08008100e800516388000600fc001202800032
:107b1800020eb30012028800716380008100e90040
:107b2800716388000600fc0011028000f141b20078
:107b380011028800f00fb20000000600edff3700c8
:107b48005268ef002ca3ef00d0e2a800d0c2a80032
:107b5800f10f2e000034800080806000006021005a
:107b680001007000003488008680a90080ff2f0083
:107b7800ae00b6006000b300700588008220a9003e
:107b88009680a800b0002000704288005028ef00be
:107b980000cf2900801f780090cf2900801f78002f
:107ba80050d02900801f780068e50700e687570055
:087bb8000000060000000600b9
:020000040000fa
:107bc000f03fb1000180b10006003500ee0309006e
:107bd00000000000403fb1000180b100fbff3d000c
:107be0001000b000203fb000020035000080090006
:087bf000000000000000060087
:020000040000fa
:107bf8000004e000060032000040e900cc82a80042
:107c0800cc82a9000040e900e14f4000fbff3a00a8
:0c7c18000000000000000000000006005a
:020000040000fa
:020000040001f9
:0457f400fffc0000b6
:020000040000fa
:020000040001f9
:0457f8009e190000f6
:020000040000fa
:020000040001f9
:0457fc007f3f0000eb
:00000001FF
